:020000040000FA
:0408000098EF0BF072
:1008100003B275EF05F0F2B493EF05F09EB09BEFD5
:1008200005F09EB2A3EF05F0F2A81AEF04F0F2B2C1
:1008300023EF04F0F2B01FEF04F047EF0BF0F29655
:10084000F29047EF0BF0CD90F2929EA02DEF04F0C6
:100850000101533F2DEF04F0542BB2C1B6F1B3C1E7
:10086000B7F1B4C1B8F1B5C1B9F1AEC1B2F1AFC120
:10087000B3F1B0C1B4F1B1C1B5F1AAC1AEF1ABC130
:10088000AFF1ACC1B0F1ADC1B1F1A6C1AAF1A7C140
:10089000ABF1A8C1ACF1A9C1ADF1A2C1A6F1A3C150
:1008A000A7F1A4C1A8F1A5C1A9F19EC1A2F19FC160
:1008B000A3F1A0C1A4F1A1C1A5F19AC19EF19BC170
:1008C0009FF19CC1A0F19DC1A1F1CECF9AF1CFCFF4
:1008D0009BF153C19CF154C19DF1CF6ACE6A0101D5
:1008E000536B546B9E90CD800FBC0F8E0FBA7CEF74
:1008F00004F00F8A47EF0BF013880F8C0FBEB9EF8F
:1009000004F09AC19EF19BC19FF19CC1A0F19DC1D1
:10091000A1F19EC1A2F19FC1A3F1A0C1A4F1A1C107
:10092000A5F1A2C1A6F1A3C1A7F1A4C1A8F1A5C1D7
:10093000A9F1A6C1AAF1A7C1ABF1A8C1ACF1A9C1A7
:10094000ADF1AAC1AEF1ABC1AFF1ACC1B0F1ADC177
:10095000B1F1AEC1B2F1AFC1B3F1B0C1B4F1B1C147
:10096000B5F1B2C1B6F1B3C1B7F1B4C1B8F1B5C117
:10097000B9F101015E6B5F6B606B616B9A515E2731
:100980009B515F239C5160239D5161239E515E27A3
:100990009F515F23A0516023A1516123A2515E2783
:1009A000A3515F23A4516023A5516123A6515E2763
:1009B000A7515F23A8516023A9516123AA515E2743
:1009C000AB515F23AC516023AD516123AE515E2723
:1009D000AF515F23B0516023B1516123B2515E2703
:1009E000B3515F23B4516023B5516123B6515E27E3
:1009F000B7515F23B8516023B9516123D8900101E9
:100A0000613360335F335E33D8900101613360330B
:100A10005F335E33D8900101613360335F335E33FF
:100A200000C10CF101C10DF102C10EF103C10FF1C2
:100A300004C110F105C111F106C112F107C113F192
:100A400008C114F109C115F10AC116F10BC117F162
:100A500034C135F111B838EF05F00101620E046FB1
:100A6000010E056F000E066F000E076F41EF05F0D7
:100A70000101A70E046F020E056F000E066F000E37
:100A8000076F5EC100F15FC101F160C102F161C198
:100A900003F182EC30F003BF04D01CBE02D01CA0D6
:100AA000108C11A059EF05F010BA59EF05F00F8026
:100AB000108A0CC100F10DC101F10EC102F10FC18C
:100AC00003F110C104F111C105F112C106F113C106
:100AD00007F114C108F115C109F116C10AF117C1D6
:100AE0000BF135C134F147EF0BF00392ABB2AB9889
:100AF000AB88030103EE00F080517F0BE92604C0B0
:100B0000EFFF802B8151805D700BD8A48B82000099
:100B10008051815D700BD8A48B9281518019D8B41B
:100B2000079047EF0BF0F2940101453F47EF0BF0C0
:100B3000462B47EF0BF09E900101533F47EF0BF020
:100B4000542B47EF0BF09E9211B843EF08F00400CE
:100B500066A1ABEF05F08BB4B5EF05F010ACB5EFC7
:100B600005F08B84109CB6EF05F08B94077C07ACE6
:100B7000D1EF05F0C274C2B4CBEF05F0C3CFB7F527
:100B8000C4CFB8F50501D890B833B733D890B8338F
:100B9000B733D2EF05F0C3CF55F1C4CF56F1D2EF42
:100BA00005F0C28207B444EF06F047C14BF148C1DB
:100BB0004CF149C14DF14AC14EF15EC162F15FC1D4
:100BC00063F160C164F161C165F113A8EAEF05F05A
:100BD000138C13989AC1BAF19BC1BBF19CC1BCF1B3
:100BE0009DC1BDF19EC1BEF19FC1BFF1A0C1C0F1C9
:100BF000A1C1C1F1A2C1C2F1A3C1C3F1A4C1C4F199
:100C0000A5C1C5F1A6C1C6F1A7C1C7F1A8C1C8F168
:100C1000A9C1C9F1AAC1CAF1ABC1CBF1ACC1CCF138
:100C2000ADC1CDF1AEC1CEF1AFC1CFF1B0C1D0F108
:100C3000B1C1D1F1B2C1D2F1B3C1D3F1B4C1D4F1D8
:100C4000B5C1D5F1B6C1D6F1B7C1D7F1B8C1D8F1A8
:100C5000B9C1D9F1B7C5B9F5B8C5BAF5B9C5BBF5CC
:100C6000BAC5BCF5010155515B2756515C23E86AB2
:100C70005D230E2E44EF06F05CC157F15DC158F1C3
:100C80005B6B5C6B5D6B078E0201002F47EF0BF017
:100C90003C0E006F1D50E00BE00AE86612881BBE98
:100CA00002D01BB4108E00C10CF101C10DF102C1C4
:100CB0000EF103C10FF104C110F105C111F106C11C
:100CC00012F107C113F108C114F109C115F10AC1EC
:100CD00016F10BC117F134C135F181AAACEF06F062
:100CE00015A4F7EF06F005012F51000AD8B43AEF2A
:100CF00007F005012F51010AD8B4B6EF06F005013F
:100D00002F51020AD8B4F7EF06F005012F51030A5C
:100D1000D8B4F7EF06F005012F51040AD8B4F7EF65
:100D200006F005012F51050AD8B4F7EF06F00501CA
:100D30002F51060AD8B4F7EF06F005012F51070A24
:100D4000D8B4F7EF06F005012F51320AD8B4B4EF4A
:100D500006F02F6B3AEF07F000011650030AD8B4E3
:100D6000F7EF06F03AEF07F03AEF07F005015767A3
:100D7000C1EF06F05867C1EF06F05967C1EF06F002
:100D80005A67C5EF06F03AEF07F05BC500F15CC5A6
:100D900001F15DC502F15EC503F10101010E046FB1
:100DA000000E056F000E066F000E076F82EC30F02C
:100DB00000C15BF501C15CF502C15DF503C15EF5E3
:100DC00001010067EBEF06F00167EBEF06F0026749
:100DD000EBEF06F003673AEF07F057C55BF558C530
:100DE0005CF559C55DF55AC55EF524EF07F00FBEF9
:100DF0000CEF07F010A011EF07F00101476708EFB3
:100E000007F0486708EF07F0496708EF07F04A67FF
:100E10000CEF07F011EF07F007AE11EF07F024EF2A
:100E200007F00501312F3AEF07F03C0E316F302FFC
:100E30003AEF07F00101000E626FE00E636FA50E3E
:100E4000646F010E656F138800011650000AD8B454
:100E500032EF07F000011650030AD8B437EF07F05D
:100E60003AEF07F00001010E166E3AEF07F00001AD
:100E7000040E166E0501666B37B740EF07F066810A
:100E80000CC100F10DC101F10EC102F10FC103F15E
:100E900010C104F111C105F112C106F113C107F12E
:100EA00014C108F115C109F116C10AF117C10BF1FE
:100EB00035C134F100C10CF101C10DF102C10EF1D7
:100EC00003C10FF104C110F105C111F106C112F106
:100ED00007C113F108C114F109C115F10AC116F1D6
:100EE0000BC117F134C135F101018E677FEF07F0B7
:100EF0008F677FEF07F090677FEF07F0916783EFD1
:100F000007F0B4EF07F092C100F193C101F194C171
:100F100002F195C103F10101010E046F000E056F8E
:100F2000000E066F000E076F82EC30F000C192F1E8
:100F300001C193F102C194F103C195F10101006770
:100F4000A9EF07F00167A9EF07F00267A9EF07F023
:100F50000367B4EF07F08EC192F18FC193F190C196
:100F600094F191C195F10F80D57ED5BE6ED0D6CFCC
:100F700047F1D7CF48F145C149F1E86AE8CF4AF1D6
:100F8000138A1CBE02D01CA0108C109047C100F127
:100F900048C101F149C102F14AC103F101010A0E40
:100FA000046F000E056F000E066F000E076F82ECD7
:100FB00030F003AF1080010154A7EBEF07F00F9A58
:100FC0000F9C0F9E0101000E5E6F600E5F6F3D0E65
:100FD000606F080E616F010147BFFBEF07F04867C4
:100FE000FBEF07F04967FBEF07F04A67FBEF07F0FD
:100FF000F28820EF08F0F2985E6B5F6B606B616BBC
:101000009A6B9B6B9C6B9D6B9E6B9F6BA06BA16B9C
:10101000A26BA36BA46BA56BA66BA76BA86BA96B4C
:10102000AA6BAB6BAC6BAD6BAE6BAF6BB06BB16BFC
:10103000B26BB36BB46BB56BB66BB76BB86BB96BAC
:10104000D76AD66A0101456B466B0CC100F10DC130
:1010500001F10EC102F10FC103F110C104F111C180
:1010600005F112C106F113C107F114C108F115C150
:1010700009F116C10AF117C10BF135C134F147EF7F
:101080000BF047EF0BF00201002FABEF0AF0D59EFB
:10109000D6CF47F1D7CF48F145C149F1E86AE8CF4B
:1010A0004AF1138AD76AD66A0101456B466BD58E21
:1010B0001D50E00BE00AE86612881BBE02D01BB48C
:1010C000108E1AAE1F8C00C10CF101C10DF102C1CE
:1010D0000EF103C10FF104C110F105C111F106C1F8
:1010E00012F107C113F108C114F109C115F10AC1C8
:1010F00016F10BC117F134C135F10FA0109A11B8D8
:101100008DEF08F00101620E046F010E056F000EF5
:10111000066F000E076F96EF08F00101A70E046F2F
:10112000020E056F000E066F000E076F47C100F13B
:1011300048C101F149C102F14AC103F182EC30F02A
:1011400003BFA9EF08F01CBE02D01CA0108C11B088
:101150000F800CC100F10DC101F10EC102F10FC1F0
:1011600003F110C104F111C105F112C106F113C15F
:1011700007F114C108F115C109F116C10AF117C12F
:101180000BF135C134F102013C0E006F00C10CF1CE
:1011900001C10DF102C10EF103C10FF104C110F143
:1011A00005C111F106C112F107C113F108C114F113
:1011B00009C115F10AC116F10BC117F134C135F19E
:1011C00081BAE6EF08F015B225EF09F015A025EF7A
:1011D00009F015A470EF09F005012F51000AD8B4E9
:1011E000B3EF09F005012F51010AD8B42FEF09F030
:1011F00005012F51020AD8B470EF09F005012F51F3
:10120000030AD8B470EF09F005012F51040AD8B4CD
:1012100070EF09F005012F51050AD8B470EF09F0FD
:1012200005012F51060AD8B470EF09F005012F51BE
:10123000070AD8B470EF09F005012F51320AD8B46B
:101240002DEF09F02F6BB3EF09F000011650030AE0
:10125000D8B470EF09F0B3EF09F0B3EF09F005016E
:1012600057673AEF09F058673AEF09F059673AEFD4
:1012700009F05A673EEF09F0B3EF09F05BC500F1E2
:101280005CC501F15DC502F15EC503F10101010E0E
:10129000046F000E056F000E066F000E076F82ECE4
:1012A00030F000C15BF501C15CF502C15DF503C121
:1012B0005EF50101006764EF09F0016764EF09F072
:1012C000026764EF09F00367B3EF09F057C55BF5F8
:1012D00058C55CF559C55DF55AC55EF59DEF09F039
:1012E0000FBE85EF09F010A08AEF09F001014767F2
:1012F00081EF09F0486781EF09F0496781EF09F054
:101300004A6785EF09F08AEF09F007AE8AEF09F026
:101310009DEF09F00501312FB3EF09F03C0E316F5D
:10132000302FB3EF09F00101000E626FE00E636F22
:10133000A50E646F010E656F138800011650000A38
:10134000D8B4ABEF09F000011650030AD8B4B0EFDF
:1013500009F0B3EF09F00001010E166EB3EF09F0CA
:101360000001040E166E0501666B37B7B9EF09F080
:1013700066810CC100F10DC101F10EC102F10FC176
:1013800003F110C104F111C105F112C106F113C13D
:1013900007F114C108F115C109F116C10AF117C10D
:1013A0000BF135C134F100C10CF101C10DF102C1E5
:1013B0000EF103C10FF104C110F105C111F106C115
:1013C00012F107C113F108C114F109C115F10AC1E5
:1013D00016F10BC117F134C135F101018E67F8EF39
:1013E00009F08F67F8EF09F09067F8EF09F091675F
:1013F000FCEF09F02DEF0AF092C100F193C101F169
:1014000094C102F195C103F10101010E046F000EB8
:10141000056F000E066F000E076F82EC30F000C102
:1014200092F101C193F102C194F103C195F101015F
:10143000006722EF0AF0016722EF0AF0026722EF4D
:101440000AF003672DEF0AF08EC192F18FC193F17C
:1014500090C194F191C195F10F80109047C100F1B6
:1014600048C101F149C102F14AC103F101010A0E6B
:10147000046F000E056F000E066F000E076F82EC02
:1014800030F003AF1080010154A753EF0AF00F9A18
:101490000F9C0F9E0101000E5E6F600E5F6F3D0E90
:1014A000606F080E616F47C100F148C101F149C189
:1014B00002F14AC103F10101140E046F050E056F1C
:1014C000000E066F000E076F82EC30F003AF6CEF7A
:1014D0000AF0F28891EF0AF0F2985E6B5F6B606B36
:1014E000616B9A6B9B6B9C6B9D6B9E6B9F6BA06BF8
:1014F000A16BA26BA36BA46BA56BA66BA76BA86B70
:10150000A96BAA6BAB6BAC6BAD6BAE6BAF6BB06B1F
:10151000B16BB26BB36BB46BB56BB66BB76BB86BCF
:10152000B96B0CC100F10DC101F10EC102F10FC187
:1015300003F110C104F111C105F112C106F113C18B
:1015400007F114C108F115C109F116C10AF117C15B
:101550000BF135C134F104008BB4B6EF0AF010ACD6
:10156000B6EF0AF08B84109CB7EF0AF08B94077CDF
:1015700007ACD2EF0AF0C274C2B4CCEF0AF0C3CF0A
:10158000B7F5C4CFB8F50501D890B833B733D890C4
:10159000B833B733D3EF0AF0C3CF55F1C4CF56F108
:1015A000D3EF0AF0C28207B445EF0BF047C14BF10D
:1015B00048C14CF149C14DF14AC14EF15EC162F1E1
:1015C0005FC163F160C164F161C165F113A8EBEF24
:1015D0000AF0138C13989AC1BAF19BC1BBF19CC15C
:1015E000BCF19DC1BDF19EC1BEF19FC1BFF1A0C1C3
:1015F000C0F1A1C1C1F1A2C1C2F1A3C1C3F1A4C193
:10160000C4F1A5C1C5F1A6C1C6F1A7C1C7F1A8C162
:10161000C8F1A9C1C9F1AAC1CAF1ABC1CBF1ACC132
:10162000CCF1ADC1CDF1AEC1CEF1AFC1CFF1B0C102
:10163000D0F1B1C1D1F1B2C1D2F1B3C1D3F1B4C1D2
:10164000D4F1B5C1D5F1B6C1D6F1B7C1D7F1B8C1A2
:10165000D8F1B9C1D9F1B7C5B9F5B8C5BAF5B9C5A9
:10166000BBF5BAC5BCF5010155515B2756515C234A
:10167000E86A5D230E2E45EF0BF05CC157F15DC1AA
:1016800058F15B6B5C6B5D6B078E47EF0BF002C034
:10169000E0FF005001C0D8FF1000A6B24DEF0BF0E4
:1016A0000CC0A9FF0BC0A8FFA69EA69CA684F29E14
:1016B000550EA76EAA0EA76EA682F28EA694A6B2AB
:1016C0005FEF0BF00C2A1200A96EA69EA69CA680C6
:1016D000A8500C2A120004012C0E826F96EC0EF01A
:1016E00097EC31F00C5064EC0BF0E8CF00F10C50AB
:1016F00064EC0BF0E8CF01F101AF84EF0BF00101D6
:10170000FF0E026FFF0E036F20EC31F0296790EFA0
:101710000BF00401200E826F96EC0EF095EF0BF0AB
:1017200004012D0E826F96EC0EF02AEC2FF01200C1
:1017300015941596076A0F6A106A116A126A136A7D
:10174000166A0F010D0EC16E860EC06E030EC26EBC
:101750000F01680E896E130E926E080E8A6EF30EDC
:10176000936E8B6A900E946EC80E64EC0BF0E8CF0B
:10177000E8FF1098E8A0108810A805D00E0E256E7E
:101780008E0E266E04D00F0E256E8F0E266E2FEC59
:1017900032F07AEC33F0F18EF19EFC0E64EC0BF03B
:1017A000E8CF0BF00BA011800BA211820BA41184C7
:1017B0000BA81188C90E64EC0BF0E8CF1AF0CA0E22
:1017C00064EC0BF0E8CF1BF0CB0E64EC0BF0E8CF31
:1017D0001CF0CC0E64EC0BF0E8CF1DF0FB0E64ECBB
:1017E0000BF0E8CF37F0CE0E64EC0BF0E8CF14F03E
:1017F000CD0E64EC0BF0E8CF36F01F6A206A0E6A5B
:1018000001015B6B5C6B5D6B576B586BF29A01016E
:10181000476B486B496B4A6B4B6B4C6B4D6B4E6B1C
:101820004F6B506B516B526B456B466BD76AD66AE8
:101830000F01280ED56EF28A9D90B00ECD6E01017B
:101840005E6B5F6B606B616B626B636B646B656B34
:10185000666B676B686B696B536B546BCF6ACE6A50
:101860000F9A0F9C0F9E9D80760ECA6E9D8202017C
:101870003C0E006FCC6A160E64EC0BF0E8CF00F162
:10188000170E64EC0BF0E8CF01F1180E64EC0BF0CE
:10189000E8CF02F1190E64EC0BF0E8CF03F101017F
:1018A00003AF6DEF0CF097EC31F0160E0C6E00C12B
:1018B0000BF04DEC0BF0170E0C6E01C10BF04DEC64
:1018C0000BF0180E0C6E02C10BF04DEC0BF0190E64
:1018D0000C6E03C10BF04DEC0BF000C18EF101C199
:1018E0008FF102C190F103C191F100C192F101C1E8
:1018F00093F102C194F103C195F11A0E64EC0BF05F
:10190000E8CF00F11B0E64EC0BF0E8CF01F11C0EE8
:1019100064EC0BF0E8CF02F11D0E64EC0BF0E8CFA5
:1019200003F1010103AFC3EF0CF097EC31F01A0E95
:101930000C6E00C10BF04DEC0BF01B0E0C6E01C1D8
:101940000BF04DEC0BF01C0E0C6E02C10BF04DECCD
:101950000BF01D0E0C6E03C10BF04DEC0BF01A0ECC
:1019600064EC0BF0E8CF00F11B0E64EC0BF0E8CF59
:1019700001F11C0E64EC0BF0E8CF02F11D0E64ECDB
:101980000BF0E8CF03F100C196F101C197F102C15C
:1019900098F103C199F1240EAC6E900EAB6E240E3B
:1019A000AC6E080EB86E000EB06E1F0EAF6E040166
:1019B000806B816B0F01900EAB6E0F019D8A03014E
:1019C000806B816BC26B8B92D4EC36F0D4EC36F02A
:1019D000B6EC38F0B2EC34F0200E64EC0BF0E8CF4B
:1019E0002FF505012F51FF0AD8A4FEEF0CF02F6B45
:1019F000200E0C6E2FC50BF04DEC0BF00501010E07
:101A0000306F3C0E316F250E64EC0BF0E8CF00F127
:101A1000260E64EC0BF0E8CF01F1270E64EC0BF01E
:101A2000E8CF02F1280E64EC0BF0E8CF03F10101DE
:101A300003AF35EF0DF097EC31F0250E0C6E00C1C1
:101A40000BF04DEC0BF0260E0C6E01C10BF04DECC3
:101A50000BF0270E0C6E02C10BF04DEC0BF0280EB4
:101A60000C6E03C10BF04DEC0BF000C157F501C13A
:101A700058F502C159F503C15AF500C15BF501C122
:101A80005CF502C15DF503C15EF5290E64EC0BF057
:101A9000E8CF5FF5050160515F5DD8A05FC560F5D7
:101AA000210E64EC0BF0E8CF00F1220E64EC0BF099
:101AB000E8CF01F1230E64EC0BF0E8CF02F1240E25
:101AC00064EC0BF0E8CF03F1010103AF96EF0DF0EA
:101AD00097EC31F0210E0C6E00C10BF04DEC0BF0C9
:101AE000220E0C6E01C10BF04DEC0BF0230E0C6EB0
:101AF00002C10BF04DEC0BF0240E0C6E03C10BF089
:101B00004DEC0BF0210E64EC0BF0E8CF00F1220E4F
:101B100064EC0BF0E8CF01F1230E64EC0BF0E8CF9E
:101B200002F1240E64EC0BF0E8CF03F100C161F583
:101B300001C162F502C163F503C164F5FAEC33F04B
:101B4000E0EC32F038EC32F01590C70E64EC0BF09C
:101B5000E8CF00F1010100B1B1EF0DF01592B2EF45
:101B60000DF0158281AAC0EF0DF015B4BBEF0DF09A
:101B70001580C0EF0DF0F5EC38F015A05CEF39F0F2
:101B800007900001F28EF28C12AE03D012BC6EEF01
:101B900019F007B0A9EF2DF00FB099EF26F010BEA5
:101BA00099EF26F012B899EF26F000011650010ABD
:101BB000D8B4A1EF1DF081BAE6EF0DF00001165088
:101BC000040AD8B41AEF1CF0ECEF0DF00001165027
:101BD000040AD8B4DDEF1DF00301805181197F0B99
:101BE000D8B4A9EF2DF013EE00F081517F0BE12660
:101BF000812BE7CFE8FFE00BD8B4A9EF2DF023EE5F
:101C000082F0C2513F0BD926E7CFDFFFC22BDF5056
:101C1000780AD8A4A9EF2DF0078092C100F193C1F2
:101C200001F194C102F195C103F10101040E046FA9
:101C3000000E056F000E066F000E076F82EC30F08D
:101C400000AF2CEF0EF00101030E926F000E936FA8
:101C5000000E946F000E956F03018251720AD8B482
:101C60001AEF26F08251520AD8B41AEF26F08251A8
:101C7000750AD8B41AEF26F08251680AD8B4AAEFD0
:101C80000EF08251630AD8B463EF2AF08251690AD8
:101C9000D8B4E7EF20F082517A0AD8B4FAEF21F0F5
:101CA0008251490AD8B486EF20F08251500AD8B444
:101CB000A4EF1FF08251700AD8B4E7EF1FF08251F1
:101CC000540AD8B412EF20F08251740AD8B458EFF5
:101CD00020F08251410AD8B4AFEF0FF082514B0A85
:101CE000D8B4ACEF0EF082516D0AD8B41FEF14F0E7
:101CF00082514D0AD8B438EF14F08251730AD8B427
:101D00004AEF25F08251530AD8B4AFEF25F0825143
:101D10004C0AD8B4C7EF14F08251590AD8B470EF06
:101D200013F012AE01D0128C9AEF2AF0040114EED7
:101D300000F080517F0BE12682C4E7FF802B120068
:101D400004010D0E826F96EC0EF00A0E826F96EC77
:101D50000EF0120098EF2AF004014B0E826F96EC01
:101D60000EF004012C0E826F96EC0EF081B802D0BA
:101D700036B630D003018351430AD8B4F1EF0EF0E8
:101D800003018351630AD8B4F3EF0EF003018351CA
:101D9000520AD8B4F5EF0EF003018351720AD8B499
:101DA000F7EF0EF003018351470AD8B4F9EF0EF0B4
:101DB00003018351670AD8B4FBEF0EF0030183518E
:101DC000540AD8B4FDEF0EF003018351740AD8B45D
:101DD0006DEF0FF003018351550AD8B4FFEF0EF0F9
:101DE00083D036807BD0369079D0368277D03692C9
:101DF00075D0368473D0369471D036866FD084C354
:101E000030F185C331F186C332F187C333F101016B
:101E1000296BE5EC31F05CEC31F000C104F101C15B
:101E200005F102C106F103C107F1D8EC31F0200E33
:101E3000F86EF76AF66A0900F5CF2CF10900F5CFC4
:101E40002DF10900F5CF2EF10900F5CF2FF1090092
:101E5000F5CF30F10900F5CF31F10900F5CF32F1BE
:101E60000900F5CF33F10101296BE5EC31F05CECB1
:101E700031F082EC30F00101006746EF0FF00167AE
:101E800046EF0FF0026746EF0FF0036701D025D051
:101E900004014E0E826F96EC0EF004016F0E826FFD
:101EA00096EC0EF004014D0E826F96EC0EF00401DC
:101EB000610E826F96EC0EF00401740E826F96EC48
:101EC0000EF00401630E826F96EC0EF00401680EB2
:101ED000826F96EC0EF098EF2AF03696CD0E0C6ECF
:101EE00036C00BF04DEC0BF0CD0E64EC0BF0E8CFF0
:101EF00036F036B006D00401630E826F96EC0EF019
:101F000005D00401430E826F96EC0EF036B206D077
:101F10000401720E826F96EC0EF005D00401520E91
:101F2000826F96EC0EF036B406D00401670E826F15
:101F300096EC0EF005D00401470E826F96EC0EF081
:101F400036B606D00401740E826F96EC0EF005D002
:101F50000401540E826F96EC0EF098EF2AF0040103
:101F6000410E826F96EC0EF003018351310AD8B412
:101F700090EF12F003018351320AD8B4C0EF11F090
:101F800003018351330AD8B449EF11F0030183519F
:101F9000340AD8B439EF10F003018351350AD8B4AC
:101FA000D9EF0FF004013F0E826F96EC0EF098EF20
:101FB0002AF003018451300AD8B4FFEF0FF0030177
:101FC0008451310AD8B402EF10F003018451650A3C
:101FD000D8B4F3EF0FF003018451640AD8B4F6EFDC
:101FE0000FF003EF10F03790F7EF0FF03780FB0E94
:101FF0000C6E37C00BF04DEC0BF003EF10F08B9034
:1020000003EF10F08B800401350E826F96EC0EF01A
:1020100004012C0E826F96EC0EF08BB017EF10F0CF
:102020000401300E826F96EC0EF01CEF10F00401EC
:10203000310E826F96EC0EF004012C0E826F96EC3E
:102040000EF0FB0E64EC0BF0E8CF37F037A030EF6A
:1020500010F00401640E826F96EC0EF035EF10F074
:102060000401650E826F96EC0EF037EF10F098EFDA
:102070002AF0CC0E64EC0BF0E8CF0BF004012C0E30
:10208000826F96EC0EF003018451310AD8B45DEFF3
:1020900010F003018451300AD8B45FEF10F003014F
:1020A00084514D0AD8B469EF10F003018451540AE9
:1020B000D8B470EF10F087EF10F08A8401D08A94C2
:1020C0000BAE04D00BAC02D00BBA21D0E00E0B1239
:1020D00018D01F0E0B168539E844E00B0B1211D0F7
:1020E000E00E0B16D8EC31F085C332F186C333F124
:1020F0000101296BE5EC31F05CEC31F000511F0B74
:102100000B12CC0E0C6E0BC00BF04DEC0BF004015F
:10211000340E826F96EC0EF004012C0E826F96EC5A
:102120000EF0CC0E64EC0BF0E8CF1DF08AB406D0B4
:102130000401300E826F96EC0EF005D00401310ED2
:10214000826F96EC0EF004012C0E826F96EC0EF06E
:102150001D38E840070BE8CF82F40401300E8227D7
:1021600096EC0EF004012C0E826F96EC0EF097ECBC
:1021700031F01D501F0BE8CF00F120EC31F032C1DF
:1021800082F40401300E822796EC0EF033C182F403
:102190000401300E822796EC0EF004012C0E826FA3
:1021A00096EC0EF097EC31F030C000F100AF0BD0A0
:1021B000FF0E016FFF0E026FFF0E036F04012D0E65
:1021C000826F96EC0EF020EC31F031C182F4040104
:1021D000300E822796EC0EF032C182F40401300EEC
:1021E000822796EC0EF033C182F40401300E822770
:1021F00096EC0EF004012C0E826F96EC0EF097EC2C
:1022000031F02FC000F120EC31F031C182F4040133
:10221000300E822796EC0EF032C182F40401300EAB
:10222000822796EC0EF033C182F40401300E82272F
:1022300096EC0EF004012C0E826F96EC0EF097ECEB
:1022400031F031C000F100AF0BD0FF0E016FFF0E77
:10225000026FFF0E036F04012D0E826F96EC0EF0DD
:1022600020EC31F031C182F40401300E822796EC6B
:102270000EF032C182F40401300E822796EC0EF08B
:1022800033C182F40401300E822796EC0EF098EFF1
:102290002AF0CB0E64EC0BF0E8CF0BF004012C0E0F
:1022A000826F96EC0EF003018451450AD8B46DEFAD
:1022B00011F003018451440AD8B470EF11F0030106
:1022C0008451300AD8B473EF11F003018451310AFC
:1022D000D8B477EF11F082EF11F00B9E7CEF11F084
:1022E0000B8E7CEF11F0FC0E0B167CEF11F0FC0E48
:1022F0000B160B807CEF11F0CB0E0C6E0BC00BF0AD
:102300004DEC0BF00401330E826F96EC0EF00401DD
:102310002C0E826F96EC0EF0CB0E64EC0BF0E8CF37
:102320001CF01CBE9BEF11F00401450E826F96EC71
:102330000EF0A0EF11F00401440E826F96EC0EF047
:1023400004012C0E826F96EC0EF00401300E826FA9
:1023500096EC0EF004012C0E826F96EC0EF01CB081
:10236000B9EF11F00401300E826F96EC0EF0BEEF63
:1023700011F00401310E826F96EC0EF098EF2AF006
:10238000CA0E64EC0BF0E8CF0BF004012C0E826F48
:1023900096EC0EF003018451450AD8B4FCEF11F01D
:1023A00003018451440AD8B4FFEF11F003018451B2
:1023B0004D0AD8B408EF12F003018451410AD8B491
:1023C00002EF12F003018451460AD8B405EF12F06F
:1023D00003018451560AD8B410EF12F0030184515E
:1023E000500AD8B41BEF12F003018451520AD8B43A
:1023F0001EEF12F027EF12F00B9E21EF12F00B8E62
:1024000021EF12F00B9C21EF12F00B8C21EF12F058
:10241000FC0E0B1685C3E8FF030B0B1221EF12F025
:10242000C70E0B1685C3E8FF070BE846E846E846EB
:102430000B1221EF12F00B8421EF12F00B9421EF1D
:1024400012F0CA0E0C6E0BC00BF04DEC0BF0CA0E66
:1024500064EC0BF0E8CF1BF00401320E826F96ECB7
:102460000EF004012C0E826F96EC0EF01BBE40EFB6
:1024700012F00401450E826F96EC0EF045EF12F05B
:102480000401440E826F96EC0EF004012C0E826F54
:1024900096EC0EF01BC0E8FF030BE8CF82F40401BA
:1024A000300E822796EC0EF004012C0E826F96EC13
:1024B0000EF01BBC63EF12F00401410E826F96EC2C
:1024C0000EF068EF12F00401460E826F96EC0EF0EB
:1024D00004012C0E826F96EC0EF01BC0E8FF380B47
:1024E000E842E842E842E8CF82F40401300E822755
:1024F00096EC0EF004012C0E826F96EC0EF01BB4DD
:1025000089EF12F00401520E826F96EC0EF08EEFFE
:1025100012F00401500E826F96EC0EF098EF2AF044
:10252000C90E64EC0BF0E8CF0BF004012C0E826FA7
:1025300096EC0EF003018451450AD8B4AEEF12F0C8
:1025400003018451440AD8B4B1EF12F0030184515D
:102550004D0AD8B4B4EF12F0C2EF12F00B9EBCEFEC
:1025600012F00B8EBCEF12F0F80E0B1685C3E8FFCD
:10257000070B0B12BCEF12F0C90E0C6E0BC00BF068
:102580004DEC0BF00401310E826F96EC0EF004015D
:102590002C0E826F96EC0EF0C90E64EC0BF0E8CFB7
:1025A0001AF01ABE06D00401450E826F96EC0EF0AA
:1025B00005D00401440E826F96EC0EF004012C0E3F
:1025C000826F96EC0EF01AC0E8FF070BE8CF82F49A
:1025D0000401300E822796EC0EF004012C0E826F5F
:1025E00096EC0EF0078097EC31F02BC0E8FF003B33
:1025F00000430043030B20EC31F033C182F40401AB
:10260000300E822796EC0EF004012C0E826F96ECB1
:102610000EF097EC31F02BC001F1019F019D2CC011
:1026200000F1010120EC31F02FC182F40401300EE1
:10263000822796EC0EF030C182F40401300E82271E
:1026400096EC0EF031C182F40401300E822796EC34
:102650000EF032C182F40401300E822796EC0EF0A7
:1026600033C182F40401300E822796EC0EF004018F
:102670002C0E826F96EC0EF097EC31F02DC001F12C
:102680002EC000F1D89001330033D89001330033CD
:10269000010120EC31F02FC182F40401300E8227B9
:1026A00096EC0EF030C182F40401300E822796ECD5
:1026B0000EF031C182F40401300E822796EC0EF048
:1026C00032C182F40401300E822796EC0EF033C141
:1026D00082F40401300E822796EC0EF098EF2AF077
:1026E000FC0E64EC0BF0E8CF0BF003018351520AAF
:1026F000D8B4A7EF13F003018351720AD8B4AAEF3C
:1027000013F003018351500AD8B4ADEF13F0030165
:102710008351700AD8B4B0EF13F003018351550A06
:10272000D8B4B3EF13F003018351750AD8B4B6EFF0
:1027300013F003018351430AD8B4BFEF13F0030130
:102740008351630AD8B4C2EF13F0CBEF13F00B90B0
:10275000C5EF13F00B80C5EF13F00B92C5EF13F02C
:102760000B82C5EF13F00B94C5EF13F00B84C5EF8C
:1027700013F00B96C5EF13F00B86C5EF13F00B9813
:10278000C5EF13F00B88C5EF13F0FC0E0C6E0BC0F9
:102790000BF04DEC0BF00401590E826F96EC0EF02D
:1027A0001190119211941198FC0E64EC0BF0E8CF8B
:1027B0000BF00BA011800BA211820BA411840BA8AB
:1027C000118811A0EBEF13F00401520E826F96EC0A
:1027D0000EF0F0EF13F00401720E826F96EC0EF023
:1027E00011A8FAEF13F00401430E826F96EC0EF07D
:1027F000FFEF13F00401630E826F96EC0EF011A24E
:1028000009EF14F00401500E826F96EC0EF00EEFFB
:1028100014F00401700E826F96EC0EF011A418EF04
:1028200014F00401550E826F96EC0EF01DEF14F0BB
:102830000401750E826F96EC0EF098EF2AF00401F9
:102840006D0E826F96EC0EF003018351300AD8B4FE
:1028500077EF14F003018351310AD8B48AEF14F0F2
:1028600003018351320AD8B49DEF14F09AEF2AF095
:1028700004014D0E826F96EC0EF0D8EC31F084C35B
:1028800031F185C332F186C333F10101296BE5ECE7
:1028900031F05CEC31F003018351300AD8B45FEFC2
:1028A00014F003018351310AD8B467EF14F0030127
:1028B0008351320AD8B46FEF14F09AEF2AF0FD0E6C
:1028C0000C6E00C10BF04DEC0BF077EF14F0FE0E28
:1028D0000C6E00C10BF04DEC0BF08AEF14F0FF0E04
:1028E0000C6E00C10BF04DEC0BF09DEF14F00401E9
:1028F000300E826F96EC0EF004012C0E826F96EC77
:102900000EF097EC31F0FD0E64EC0BF0E8CF00F127
:10291000AEEF14F00401310E826F96EC0EF004015C
:102920002C0E826F96EC0EF097EC31F0FE0E64ECFC
:102930000BF0E8CF00F1AEEF14F00401320E826F1D
:1029400096EC0EF097EC31F004012C0E826F96ECB1
:102950000EF0FF0E64EC0BF0E8CF00F120EC31F04C
:1029600031C182F40401300E822796EC0EF032C1A0
:1029700082F40401300E822796EC0EF033C182F40B
:102980000401300E822796EC0EF098EF2AF0030136
:102990008351300AD8B41BEF1AF003018351310A76
:1029A000D8B448EF1BF003018351320AD8B4B6EF14
:1029B0001BF003018351330AD8B4C6EF1BF00301A7
:1029C0008351340AD8B421EF1CF003018351350A36
:1029D000D8B4F5EF1DF003018351360AD8B423EFC4
:1029E0001EF003018351370AD8B4F3EF17F0030147
:1029F0008351380AD8B491EF18F003018351440A87
:102A0000D8B41FEF16F003018351640AD8B43FEF26
:102A100016F003018351460AD8B4FAEF1CF0030103
:102A200083514D0AD8B46CEF16F0030183516D0A3F
:102A3000D8B486EF16F0030183515A0AD8B4C2EF16
:102A40001AF003018351490AD8B423EF1FF00301A0
:102A50008351500AD8B455EF1EF003018351540A34
:102A6000D8B4CEEF1EF003018351630AD8B4A6EFA9
:102A700016F003018351430AD8B49EEF17F0030107
:102A80008351730AD8B4A4EF16F003018351610A8D
:102A9000D8B46CEF15F003018351650AD8B46BEF1D
:102AA0001AF003018351450AD8B479EF1AF00301F3
:102AB0008351620AD8B487EF1AF003018351420AA6
:102AC000D8B495EF1AF003018351760AD8B4A3EF76
:102AD0001AF0D8A49AEF2AF004014C0E826F96ECFB
:102AE0000EF00401610E826F96EC0EF0E0EC32F015
:102AF00004012C0E826F96EC0EF097EC31F0AFC50E
:102B000000F1010120EC31F031C182F40401300EFA
:102B1000822796EC0EF032C182F40401300E822737
:102B200096EC0EF033C182F40401300E822796EC4D
:102B30000EF004012C0E826F96EC0EF097EC31F043
:102B4000B0C500F1010120EC31F031C182F4040183
:102B5000300E822796EC0EF032C182F40401300E62
:102B6000822796EC0EF033C182F40401300E8227E6
:102B700096EC0EF004012C0E826F96EC0EF097ECA2
:102B800031F0B1C500F1010120EC31F031C182F426
:102B90000401300E822796EC0EF032C182F404015B
:102BA000300E822796EC0EF033C182F40401300E11
:102BB000822796EC0EF004012C0E826F96EC0EF03C
:102BC00097EC31F0B2C500F1010120EC31F031C1D8
:102BD00082F40401300E822796EC0EF032C182F4AA
:102BE0000401300E822796EC0EF033C182F404010A
:102BF000300E822796EC0EF004012C0E826F96ECBC
:102C00000EF097EC31F0B6C500F1010120EC31F087
:102C100031C182F40401300E822796EC0EF032C1ED
:102C200082F40401300E822796EC0EF033C182F458
:102C30000401300E822796EC0EF051EF1EF00301D6
:102C40008451300AD8B42BEF16F003018451310AB5
:102C5000D8B42FEF16F01592159630EF16F01582B6
:102C6000C70E64EC0BF0E8CF00F10101008115A262
:102C70000091C70E0C6E00C10BF04DEC0BF0C70EAF
:102C800064EC0BF0E8CF00F1010100B14BEF16F05E
:102C900015924CEF16F0158204014C0E826F96ECE3
:102CA0000EF00401640E826F96EC0EF004012C0EFF
:102CB000826F96EC0EF015B265EF16F00401300E3F
:102CC000826F96EC0EF06AEF16F00401310E826FFF
:102CD00096EC0EF098EF2AF0D8EC31F084C333F183
:102CE000E5EC31F05CEC31F0200E0C6E00C10BF025
:102CF0004DEC0BF000C12FF505012F51000A06E045
:102D000005012F51010A02E07AEC33F004014C0E68
:102D1000826F96EC0EF004014D0E826F96EC0EF071
:102D200004012C0E826F96EC0EF097EC31F02FC55B
:102D300000F120EC31F033C182F40401300E82271F
:102D400096EC0EF051EF1EF05CEF39F004014C0EE2
:102D5000826F96EC0EF00401630E826F96EC0EF01B
:102D600038EC32F004012C0E826F96EC0EF0BBECC6
:102D700016F051EF1EF097EC31F0B5C500F10101EE
:102D8000003B0F0E001720EC31F033C182F4040138
:102D9000300E822796EC0EF0B5C500F101010F0E42
:102DA0000101001720EC31F033C182F40401300E30
:102DB000822796EC0EF004012D0E826F96EC0EF039
:102DC000B4C500F10101003B0F0E001720EC31F0FB
:102DD00033C182F40401300E822796EC0EF0B4C5A4
:102DE00000F101010F0E0101001720EC31F033C199
:102DF00082F40401300E822796EC0EF004012D0EB1
:102E0000826F96EC0EF0B3C500F10101003B0F0E8E
:102E1000001720EC31F033C182F40401300E822718
:102E200096EC0EF0B3C500F101010F0E0101001781
:102E300020EC31F033C182F40401300E822796EC8D
:102E40000EF00401200E826F96EC0EF0B2C500F178
:102E50000F0E0101001720EC31F033C182F40401A0
:102E6000300E822796EC0EF00401200E826F96EC55
:102E70000EF0B1C500F101010101003B0F0E00177A
:102E800020EC31F033C182F40401300E822796EC3D
:102E90000EF0B1C500F101010F0E0101001720EC89
:102EA00031F033C182F40401300E822796EC0EF02B
:102EB00004013A0E826F96EC0EF0B0C500F10101EC
:102EC000003B0F0E001720EC31F033C182F40401F7
:102ED000300E822796EC0EF0B0C500F101010F0E06
:102EE0000101001720EC31F033C182F40401300EEF
:102EF000822796EC0EF004013A0E826F96EC0EF0EB
:102F0000AFC500F10101003B0F0E001720EC31F0BE
:102F100033C182F40401300E822796EC0EF0AFC567
:102F200000F101010F0E001720EC31F033C182F4E3
:102F30000401300E822796EC0EF0120084C3E8FFE5
:102F40000F0BE83AE8CFB5F585C3E8FF0F0B050195
:102F5000B51387C3E8FF0F0BE83AE8CFB4F588C391
:102F6000E8FF0F0B0501B4138AC3E8FF0F0BE83A23
:102F7000E8CFB3F58BC3E8FF0F0B0501B3138DC387
:102F8000E8FF0F0BE8CFB2F58FC3E8FF0F0BE83A6D
:102F9000E8CFB1F590C3E8FF0F0B0501B11392C361
:102FA000E8FF0F0BE83AE8CFB0F593C3E8FF0F0B4B
:102FB0000501B01395C3E8FF0F0BE83AE8CFAFF572
:102FC00096C3E8FF0F0B0501AF1393EC32F0040139
:102FD0004C0E826F96EC0EF00401430E826F96EC5D
:102FE0000EF0B0EF16F0078404014C0E826F96ECE1
:102FF0000EF00401370E826F96EC0EF004012C0ED9
:10300000826F96EC0EF005012E51130A06E00501C1
:103010002E51170A0DE08EEF18F00101000E006F1F
:10302000000E016F100E026F000E036F21EF18F0FB
:103030000101000E006F000E016F000E026F010E05
:10304000036F20EC31F02AC182F40401300E822794
:1030500096EC0EF02BC182F40401300E822796EC20
:103060000EF02CC182F40401300E822796EC0EF093
:103070002DC182F40401300E822796EC0EF02EC191
:1030800082F40401300E822796EC0EF02FC182F4F8
:103090000401300E822796EC0EF030C182F4040158
:1030A000300E822796EC0EF031C182F40401300E0E
:1030B000822796EC0EF032C182F40401300E822792
:1030C00096EC0EF033C182F40401300E822796ECA8
:1030D0000EF004012C0E826F96EC0EF00101100E22
:1030E000006F000E016F000E026F000E036F20ECE8
:1030F00031F031C182F40401300E822796EC0EF0DB
:1031000032C182F40401300E822796EC0EF033C1F6
:1031100082F40401300E822796EC0EF0079451EFF2
:103120001EF00501216B226B236B246B04014C0EF6
:10313000826F96EC0EF00401380E826F96EC0EF062
:1031400004012C0E826F96EC0EF00101100E006F40
:10315000000E016F000E026F000E036F20EC31F0C5
:103160002AC182F40401300E822796EC0EF02BC1A6
:1031700082F40401300E822796EC0EF02CC182F40A
:103180000401300E822796EC0EF02DC182F404016A
:10319000300E822796EC0EF02EC182F40401300E20
:1031A000822796EC0EF02FC182F40401300E8227A4
:1031B00096EC0EF030C182F40401300E822796ECBA
:1031C0000EF031C182F40401300E822796EC0EF02D
:1031D00032C182F40401300E822796EC0EF033C126
:1031E00082F40401300E822796EC0EF004012C0EBE
:1031F000826F96EC0EF025C500F126C501F127C5BA
:1032000002F128C503F10101100E046F000E056FD5
:10321000000E066F000E076FB3EC30F000C133F5FF
:1032200001C134F502C135F503C136F520EC31F0AA
:103230002AC182F40401300E822796EC0EF02BC1D5
:1032400082F40401300E822796EC0EF02CC182F439
:103250000401300E822796EC0EF02DC182F4040199
:10326000300E822796EC0EF02EC182F40401300E4F
:10327000822796EC0EF02FC182F40401300E8227D3
:1032800096EC0EF030C182F40401300E822796ECE9
:103290000EF031C182F40401300E822796EC0EF05C
:1032A00032C182F40401300E822796EC0EF033C155
:1032B00082F40401300E822796EC0EF0A0EC0EF0A2
:1032C000050133676BEF19F034676BEF19F0356761
:1032D0006BEF19F0366702D00AEF1AF0129E129CBB
:1032E00021C500F122C501F123C502F124C503F176
:1032F000899A400EC76E200EC66E9E96C69E0B0E15
:10330000C96EFF0E9EB602D0E82EFCD79E96C69ED2
:1033100002C1C9FFFF0E9EB602D0E82EFCD79E96D2
:10332000C69E01C1C9FFFF0E9EB602D0E82EFCD793
:103330009E96C69E00C1C9FFFF0E9EB602D0E82E23
:10334000FCD79E96C69EC952FF0E9EB602D0E82EAE
:10335000FCD70501100E326F040114EE00F080510D
:103360007F0BE1269E96C69EC952FF0E9EB602D0E6
:10337000E82EFCD7C9CFE7FF0401802B0501322FCF
:10338000ACEF19F0898A33C500F134C501F135C5B8
:1033900002F136C503F10101010E046F000E056F45
:1033A000000E066F000E076F82EC30F000C133F59F
:1033B00001C134F502C135F503C136F505013367A6
:1033C000E9EF19F03467E9EF19F03567E9EF19F023
:1033D000366702D00AEF1AF021C500F122C501F1CB
:1033E00023C502F124C503F10101100E046F000E84
:1033F000056F000E066F000E076F87EC30F000C1FE
:1034000021F501C122F502C123F503C124F5128E75
:103410009AEF2AF00401450E826F96EC0EF004013B
:103420004F0E826F96EC0EF00401460E826F96EC02
:103430000EF051EF1EF00784B6EC38F097EC31F047
:103440002DC500F120EC31F004014C0E826F96EC9A
:103450000EF00401300E826F96EC0EF004012C0E7B
:10346000826F96EC0EF031C182F40401300E822797
:1034700096EC0EF032C182F40401300E822796ECF5
:103480000EF033C182F40401300E822796EC0EF068
:1034900004012C0E826F96EC0EF097EC31F02EC5E5
:1034A00000F120EC31F031C182F40401300E8227AA
:1034B00096EC0EF032C182F40401300E822796ECB5
:1034C0000EF033C182F40401300E822796EC0EF028
:1034D000079451EF1EF004014C0E826F96EC0EF033
:1034E0000401650E826F96EC0EF056EC34F051EF4D
:1034F0001EF004014C0E826F96EC0EF00401450E96
:10350000826F96EC0EF06DEC34F051EF1EF004017A
:103510004C0E826F96EC0EF00401620E826F96ECF8
:103520000EF09BEC34F051EF1EF004014C0E826F54
:1035300096EC0EF00401420E826F96EC0EF084ECD5
:1035400034F051EF1EF004014C0E826F96EC0EF039
:103550000401760E826F96EC0EF004012C0E826F41
:1035600096EC0EF010A807D00401310E826F96EC95
:103570000EF051EF1EF00401300E826F96EC0EF04B
:1035800051EF1EF004014C0E826F96EC0EF0040118
:103590005A0E826F96EC0EF004012C0E826F96ECA0
:1035A0000EF0B6EC38F097EC31F005012E51130A0D
:1035B00006E005012E51170A0DE0F3EF1AF00101A4
:1035C000000E006F000E016F100E026F000E036FF1
:1035D000F3EF1AF00101000E006F000E016F000EF4
:1035E000026F010E036F0101100E046F000E056FD4
:1035F000000E066F000E076FB3EC30F020EC31F0D8
:103600002AC182F40401300E822796EC0EF02BC101
:1036100082F40401300E822796EC0EF02CC182F465
:103620000401300E822796EC0EF02DC182F40401C5
:10363000300E822796EC0EF02EC182F40401300E7B
:10364000822796EC0EF02FC182F40401300E8227FF
:1036500096EC0EF030C182F40401300E822796EC15
:103660000EF031C182F40401300E822796EC0EF088
:1036700032C182F40401300E822796EC0EF033C181
:1036800082F40401300E822796EC0EF051EF1EF00A
:10369000078404014C0E826F96EC0EF00401310E8B
:1036A000826F96EC0EF004012C0E826F96EC0EF0F9
:1036B00025C500F126C501F127C502F128C503F192
:1036C0000101100E046F000E056F000E066F000E54
:1036D000076FB3EC30F020EC31F02AC182F4040122
:1036E000300E822796EC0EF02BC182F40401300ECE
:1036F000822796EC0EF02CC182F40401300E822752
:1037000096EC0EF02DC182F40401300E822796EC67
:103710000EF02EC182F40401300E822796EC0EF0DA
:103720002FC182F40401300E822796EC0EF030C1D6
:1037300082F40401300E822796EC0EF031C182F43F
:103740000401300E822796EC0EF032C182F404019F
:10375000300E822796EC0EF033C182F40401300E55
:10376000822796EC0EF0079451EF1EF007840401B7
:103770004C0E826F96EC0EF00401320E826F96ECC6
:103780000EF08AEC36F0079451EF1EF0078437B044
:10379000CCEF1BF0DFEF1BF0010E166E04014C0E98
:1037A000826F96EC0EF00401330E826F96EC0EF0F1
:1037B000E7EC36F0000E166E079453EF1BF0020E86
:1037C000166EE7EC36F08B800501010E306F3C0E73
:1037D000316F01015E6B5F6B606B616B626B636B82
:1037E000646B656B666B676B686B696B536B546B73
:1037F000CF6ACE6A0F9A0F9C0F9E030E166E0401BD
:103800004C0E826F96EC0EF00401330E826F96EC34
:103810000EF004012C0E826F96EC0EF004012D0EBA
:10382000826F96EC0EF00401310E826F96EC0EF072
:1038300098EF2AF0E7EC36F0000E166E8B909AEFB8
:103840002AF0078404014C0E826F96EC0EF00401FE
:10385000340E826F96EC0EF004012C0E826F96EC03
:103860000EF0D8EC31F084C32AF185C32BF186C366
:103870002CF187C32DF188C32EF189C32FF18AC3A0
:1038800030F18BC331F18CC332F18DC333F10101BF
:10389000296BE5EC31F05CEC31F0100E046F000E9A
:1038A000056F000E066F000E076F93EC30F000C13D
:1038B00021F501C122F502C123F503C124F569EC0C
:1038C00038F038C5AFF539C5B0F53AC5B1F53BC5E7
:1038D000B2F53CC5B3F53DC5B4F53EC5B5F5BBEC99
:1038E00016F004012C0E826F96EC0EF03FC500F12D
:1038F00040C501F141C502F142C503F10101000ECD
:10390000046F000E056F010E066F000E076FB3EC1B
:1039100030F020EC31F0296790EF1CF095EF1CF0AF
:1039200004012D0E826F96EC0EF030C182F404017A
:10393000300E822796EC0EF031C182F40401300E75
:10394000822796EC0EF004012E0E826F96EC0EF09C
:1039500032C182F40401300E822796EC0EF033C19E
:1039600082F40401300E822796EC0EF004012C0E36
:10397000826F96EC0EF097EC31F043C500F144C530
:1039800001F1C4EC2BF004012C0E826F96EC0EF0CA
:1039900097EC31F045C500F120EC31F031C182F4F3
:1039A0000401300E822796EC0EF032C182F404013D
:1039B000300E822796EC0EF033C182F40401300EF3
:1039C000822796EC0EF004012C0E826F96EC0EF01E
:1039D00037C5E8FFE8B806D00401300E826F96ECD8
:1039E0000EF005D00401310E826F96EC0EF00794B4
:1039F00051EF1EF0D8EC31F085C32AF186C32BF1CC
:103A000087C32CF188C32DF189C32EF18AC32FF10E
:103A10008BC330F18CC331F18DC332F18EC333F1DE
:103A20000101296BE5EC31F05CEC31F00101010E94
:103A3000046F000E056F000E066F000E076F82EC1C
:103A400030F0100E046F000E056F000E066F000EB2
:103A5000076F93EC30F000C129F501C12AF502C1CE
:103A60002BF503C12CF511EC36F004014C0E826FDE
:103A700096EC0EF00401460E826F96EC0EF00401F7
:103A80002C0E826F96EC0EF025C500F126C501F1D3
:103A900027C502F128C503F10101100E046F000EC5
:103AA000056F000E066F000E076FB3EC30F020ECD0
:103AB00031F02AC182F40401300E822796EC0EF018
:103AC0002BC182F40401300E822796EC0EF02CC13B
:103AD00082F40401300E822796EC0EF02DC182F4A0
:103AE0000401300E822796EC0EF02EC182F4040100
:103AF000300E822796EC0EF02FC182F40401300EB6
:103B0000822796EC0EF030C182F40401300E822739
:103B100096EC0EF031C182F40401300E822796EC4F
:103B20000EF032C182F40401300E822796EC0EF0C2
:103B300033C182F40401300E822796EC0EF051EF6F
:103B40001EF037B0A6EF1DF0020E166EE7EC36F051
:103B500000011650020AD8B4C4EF1DF005012F5120
:103B6000010AD8B4BAEF1DF015B2BFEF1DF081BA4B
:103B7000BFEF1DF0000E166E15849AEF2AF0050EA9
:103B8000166E15845CEF39F08B8001015E6B5F6B04
:103B9000606B616B626B636B646B656B666B676BB1
:103BA000686B696B536B546BCF6ACE6A0F9A0F9C2C
:103BB0000F9E030E166E9AEF2AF0E7EC36F0050121
:103BC0002F51010AD8B4EBEF1DF015B2F0EF1DF044
:103BD00081BAF0EF1DF0000E166E15849AEF2AF0F0
:103BE000050E166E15845CEF39F004014C0E826FE1
:103BF00096EC0EF00401350E826F96EC0EF0040187
:103C00002C0E826F96EC0EF097EC31F00784B9C55C
:103C100000F1079420EC31F031C182F40401300E40
:103C2000822796EC0EF032C182F40401300E822716
:103C300096EC0EF033C182F40401300E822796EC2C
:103C40000EF051EF1EF0AAEC36F097EC31F037C5CC
:103C500000F120EC31F004014C0E826F96EC0EF076
:103C60000401360E826F96EC0EF004012C0E826F6A
:103C700096EC0EF031C182F40401300E822796ECEE
:103C80000EF032C182F40401300E822796EC0EF061
:103C900033C182F40401300E822796EC0EF051EF0E
:103CA0001EF0A0EC0EF09AEF2AF004014C0E826F89
:103CB00096EC0EF00401500E826F96EC0EF00401AB
:103CC0002C0E826F96EC0EF085C32AF186C32BF181
:103CD00087C32CF188C32DF189C32EF18AC32FF13C
:103CE0008BC330F18CC331F18DC332F18EC333F10C
:103CF0000101E5EC31F05CEC31F003018451530A31
:103D00000DE0030184514D0A38E00401780E826F02
:103D100096EC0EF0A0EC0EF09AEF2AF00401530E90
:103D2000826F96EC0EF0250E0C6E00C10BF04DEC80
:103D30000BF0260E0C6E01C10BF04DEC0BF0270EB4
:103D40000C6E02C10BF04DEC0BF0280E0C6E03C193
:103D50000BF04DEC0BF000C157F501C158F502C155
:103D600059F503C15AF500C15BF501C15CF502C10B
:103D70005DF503C15EF532EF1FF004014D0E826F59
:103D800096EC0EF0290E0C6E00C10BF04DEC0BF012
:103D900000C15FF500C160F532EF1FF004014C0E69
:103DA000826F96EC0EF00401540E826F96EC0EF0CA
:103DB00004012C0E826F96EC0EF084C32AF185C3A9
:103DC0002BF186C32CF187C32DF188C32EF189C353
:103DD0002FF18AC330F18BC331F18DC332F18EC321
:103DE00033F10101E5EC31F05CEC31F00101000E42
:103DF000046F000E056F010E066F000E076F93EC47
:103E000030F0210E0C6E00C10BF04DEC0BF0220EC9
:103E10000C6E01C10BF04DEC0BF0230E0C6E02C1C9
:103E20000BF04DEC0BF0240E0C6E03C10BF04DECBF
:103E30000BF000C161F501C162F502C163F503C178
:103E400064F532EF1FF004014C0E826F96EC0EF019
:103E50000401490E826F96EC0EF004012C0E826F65
:103E600096EC0EF0250E64EC0BF0E8CF00F1260E78
:103E700064EC0BF0E8CF01F1270E64EC0BF0E8CF17
:103E800002F1280E64EC0BF0E8CF03F120EC31F0E6
:103E9000E3EC2EF00401730E826F96EC0EF0040139
:103EA0002C0E826F96EC0EF097EC31F0290E64EC3C
:103EB0000BF0E8CF00F120EC31F0E3EC2EF0040140
:103EC0006D0E826F96EC0EF004012C0E826F96EC54
:103ED0000EF05BC500F15CC501F15DC502F15EC588
:103EE00003F120EC31F0E3EC2EF00401730E826F4D
:103EF00096EC0EF004012C0E826F96EC0EF097EC0F
:103F000031F060C500F120EC31F0E3EC2EF004015B
:103F10006D0E826F96EC0EF004012C0E826F96EC03
:103F20000EF061C500F162C501F163C502F164C51F
:103F300003F1B5EC2AF004012C0E826F96EC0EF022
:103F4000A0EC0EF09AEF2AF083C32AF184C32BF180
:103F500085C32CF186C32DF187C32EF188C32FF1C1
:103F600089C330F18AC331F18BC332F18CC333F191
:103F70000101E5EC31F05CEC31F0160E0C6E00C185
:103F80000BF04DEC0BF0170E0C6E01C10BF04DEC6D
:103F90000BF0180E0C6E02C10BF04DEC0BF0190E6D
:103FA0000C6E03C10BF04DEC0BF000C18EF101C1A2
:103FB0008FF102C190F103C191F100C192F101C1F1
:103FC00093F102C194F103C195F186EF20F083C310
:103FD0002AF184C32BF185C32CF186C32DF187C34D
:103FE0002EF188C32FF189C330F18AC331F18BC31D
:103FF00032F18CC333F10101E5EC31F05CEC31F0CE
:1040000000C18EF101C18FF102C190F103C191F1A4
:1040100000C192F101C193F102C194F103C195F184
:1040200086EF20F083C32AF184C32BF185C32CF1E2
:1040300086C32DF187C32EF188C32FF189C330F1D8
:104040008AC331F18CC332F18DC333F10101E5EC48
:1040500031F05CEC31F00101000E046F000E056FD1
:10406000010E066F000E076F93EC30F01A0E0C6E07
:1040700000C10BF04DEC0BF01B0E0C6E01C10BF0F0
:104080004DEC0BF01C0E0C6E02C10BF04DEC0BF066
:104090001D0E0C6E03C10BF04DEC0BF000C196F140
:1040A00001C197F102C198F103C199F186EF20F0A7
:1040B00083C32AF184C32BF185C32CF186C32DF170
:1040C00087C32EF188C32FF189C330F18AC331F140
:1040D0008CC332F18DC333F10101E5EC31F05CECBE
:1040E00031F00101000E046F000E056F010E066F26
:1040F000000E076F93EC30F000C196F101C197F10B
:1041000002C198F103C199F186EF20F0160E64EC1C
:104110000BF0E8CF00F1170E64EC0BF0E8CF01F1E3
:10412000180E64EC0BF0E8CF02F1190E64EC0BF002
:10413000E8CF03F120EC31F0E3EC2EF00401730E34
:10414000826F96EC0EF004012C0E826F96EC0EF04E
:104150008EC100F18FC101F190C102F191C103F153
:1041600020EC31F0E3EC2EF00401730E826F96EC3C
:104170000EF004012C0E826F96EC0EF01A0E64EC19
:104180000BF0E8CF00F11B0E64EC0BF0E8CF01F16F
:104190001C0E64EC0BF0E8CF02F11D0E64EC0BF08A
:1041A000E8CF03F1B5EC2AF004012C0E826F96ECF7
:1041B0000EF096C100F197C101F198C102F199C1C9
:1041C00003F1B5EC2AF0A0EC0EF09AEF2AF004010E
:1041D000690E826F96EC0EF004012C0E826F96EC45
:1041E0000EF00101040E006F000E016F000E026F51
:1041F000000E036F20EC31F02CC182F40401300E6C
:10420000822796EC0EF02DC182F40401300E822735
:1042100096EC0EF02EC182F40401300E822796EC4B
:104220000EF02FC182F40401300E822796EC0EF0BE
:1042300030C182F40401300E822796EC0EF031C1B9
:1042400082F40401300E822796EC0EF032C182F423
:104250000401300E822796EC0EF033C182F4040183
:10426000300E822796EC0EF004012C0E826F96EC35
:104270000EF00101060E006F000E016F000E026FBE
:10428000000E036F20EC31F02CC182F40401300EDB
:10429000822796EC0EF02DC182F40401300E8227A5
:1042A00096EC0EF02EC182F40401300E822796ECBB
:1042B0000EF02FC182F40401300E822796EC0EF02E
:1042C00030C182F40401300E822796EC0EF031C129
:1042D00082F40401300E822796EC0EF032C182F493
:1042E0000401300E822796EC0EF033C182F40401F3
:1042F000300E822796EC0EF004012C0E826F96ECA5
:104300000EF001014F0E006F000E016F000E026FE4
:10431000000E036F20EC31F02CC182F40401300E4A
:10432000822796EC0EF02DC182F40401300E822714
:1043300096EC0EF02EC182F40401300E822796EC2A
:104340000EF02FC182F40401300E822796EC0EF09D
:1043500030C182F40401300E822796EC0EF031C198
:1043600082F40401300E822796EC0EF032C182F402
:104370000401300E822796EC0EF033C182F4040162
:10438000300E822796EC0EF004012C0E826F96EC14
:104390000EF0200EF86EF76AF66A04010900F5CFF8
:1043A00082F496EC0EF00900F5CF82F496EC0EF054
:1043B0000900F5CF82F496EC0EF00900F5CF82F4F7
:1043C00096EC0EF00900F5CF82F496EC0EF00900A1
:1043D000F5CF82F496EC0EF00900F5CF82F496EC5E
:1043E0000EF00900F5CF82F496EC0EF0A0EC0EF082
:1043F0009AEF2AF08351630AD8A498EF2AF08451E7
:10440000610AD8A498EF2AF085516C0AD8A498EFD5
:104410002AF08651410A3FE08651440A1BE086514A
:10442000420AD8B45EEF22F08651350AD8B424EFA0
:104430002CF08651360AD8B479EF2CF08651370A21
:10444000D8B4E2EF2CF08651380AD8B440EF2DF002
:1044500098EF2AF00798079A04017A0E826F96EC7B
:104460000EF00401780E826F96EC0EF00401640EDB
:10447000826F96EC0EF00401550E826F96EC0EF0F2
:1044800047EF22F004014C0E826F96EC0EF0A0EC88
:104490000EF09AEF2AF00788079A04017A0E826FCD
:1044A00096EC0EF00401410E826F96EC0EF00401C2
:1044B000610E826F96EC0EF03BEF22F00798078AB0
:1044C00004017A0E826F96EC0EF00401420E826FA8
:1044D00096EC0EF00401610E826F96EC0EF03BEF4D
:1044E00022F0010166677CEF22F067677CEF22F023
:1044F00068677CEF22F0696716D001014F6788EF8B
:1045000022F0506788EF22F0516788EF22F052675F
:104510000AD00101000E006F000E016F000E026F45
:10452000000E036F120011B80AD00101620E046F71
:10453000010E056F000E066F000E076F09D0010116
:10454000A70E046F020E056F000E066F000E076FB8
:1045500066C100F167C101F168C102F169C103F1EF
:1045600082EC30F003BF25EF23F0119A119C01017A
:10457000000E046FA80E056F550E066F020E076F32
:1045800066C100F167C101F168C102F169C103F1BF
:1045900066C18AF167C18BF168C18CF169C18DF187
:1045A00082EC30F003BF0BD00101000E8A6FA80E21
:1045B0008B6F550E8C6F020E8D6F118A119C0E0E33
:1045C00064EC0BF0E8CF18F10F0E64EC0BF0E8CFC1
:1045D00019F1100E64EC0BF0E8CF1AF1110E64EC37
:1045E0000BF0E8CF1BF1CBEC2FF08AC104F18BC1AB
:1045F00005F18CC106F18DC107F182EC30F0078224
:104600008FEC2FF0CBEC2FF007928FEC2FF08AC1BC
:1046100000F18BC101F18CC102F18DC103F1079250
:104620008FEC2FF0CC0E046FE00E056F870E066F37
:10463000050E076F82EC30F000C118F101C119F1CD
:1046400002C11AF103C11BF140D013AA2AEF23F0D3
:10465000138E139A119C119A0101800E006F1A0E8D
:10466000016F060E026F000E036F4FC104F150C1BF
:1046700005F151C106F152C107F182EC30F003AFF0
:1046800005D097EC31F0118C119A12000E0E64ECEB
:104690000BF0E8CF18F10F0E64EC0BF0E8CF19F136
:1046A000100E64EC0BF0E8CF1AF1110E64EC0BF075
:1046B000E8CF1BF14FC100F150C101F151C102F12E
:1046C00052C103F107828FEC2FF018C100F119C11C
:1046D00001F11AC102F11BC103F112000784BAC132
:1046E00066F1BBC167F1BCC168F1BDC169F14BC1E5
:1046F0004FF14CC150F14DC151F14EC152F157C172
:1047000059F158C15AF10794010166678FEF23F000
:1047100067678FEF23F068678FEF23F0696716D024
:1047200001014F679BEF23F050679BEF23F0516728
:104730009BEF23F052670AD00101000E006F000EBC
:10474000016F000E026F000E036F120011B80AD045
:104750000101620E046F010E056F000E066F000E60
:10476000076F09D00101A70E046F020E056F000E3E
:10477000066F000E076F66C100F167C101F168C1E5
:1047800002F169C103F182EC30F003BF27EF24F09E
:104790000101000E046FA80E056F550E066F020E84
:1047A000076F66C100F167C101F168C102F169C11B
:1047B00003F166C18AF167C18BF168C18CF169C1EF
:1047C0008DF182EC30F003BF09D00101000E8A6F39
:1047D000A80E8B6F550E8C6F020E8D6FCBEC2FF0E9
:1047E00000C104F101C105F102C106F103C107F1E5
:1047F000000E006FA00E016F980E026F7B0E036F0C
:10480000B3EC30F000C118F101C119F102C11AF185
:1048100003C11BF1000E006FA00E016F980E026F16
:104820007B0E036F8AC104F18BC105F18CC106F1C7
:104830008DC107F1B3EC30F018C104F119C105F1D5
:104840001AC106F11BC107F182EC30F01200010120
:10485000A80E006F610E016F000E026F000E036F55
:104860004FC104F150C105F151C106F152C107F128
:1048700082EC30F003AF0AD00101A80E006F610E88
:10488000016F000E026F000E036F00D0C80E006FA4
:10489000AF0E016F000E026F000E036F4FC104F1E7
:1048A00050C105F151C106F152C107F193EC30F04E
:1048B00012000784BAC166F1BBC167F1BCC168F1DF
:1048C000BDC169F14BC14FF14CC150F14DC151F126
:1048D0004EC152F157C159F158C15AF10794010123
:1048E00066677AEF24F067677AEF24F068677AEFFB
:1048F00024F0696716D001014F6786EF24F05067F6
:1049000086EF24F0516786EF24F052670AD0010148
:10491000000E006F000E016F000E026F000E036F9D
:10492000120011B80AD00101620E046F010E056F6A
:10493000000E066F000E076F09D00101A70E046F6D
:10494000020E056F000E066F000E076F66C100F1C4
:1049500067C101F168C102F169C103F182EC30F075
:1049600003BF3CEF25F00101000E046FA80E056F98
:10497000550E066F020E076F66C100F167C101F1A7
:1049800068C102F169C103F166C18AF167C18BF1A7
:1049900068C18CF169C18DF182EC30F003BF09D0A0
:1049A0000101000E8A6FA80E8B6F550E8C6F020EE0
:1049B0008D6F010E006F000E016F000E026F000E72
:1049C000036F8AC104F18BC105F18CC106F18DC161
:1049D00007F1B3EC30F018C104F119C105F11AC1A7
:1049E00006F11BC107F120EC31F02AC182F4040169
:1049F000300E822796EC0EF02BC182F40401300EAB
:104A0000822796EC0EF02CC182F40401300E82272E
:104A100096EC0EF02DC182F40401300E822796EC44
:104A20000EF02EC182F40401300E822796EC0EF0B7
:104A30002FC182F40401300E822796EC0EF030C1B3
:104A400082F40401300E822796EC0EF031C182F41C
:104A50000401300E822796EC0EF032C182F404017C
:104A6000300E822796EC0EF033C182F40401300E32
:104A7000822796EC0EF012004FC100F150C101F1F7
:104A800051C102F152C103F1010120EC31F0E3EC1C
:104A90002EF012000401730E826F96EC0EF00401EA
:104AA0002C0E826F96EC0EF0078462C166F163C132
:104AB00067F164C168F165C169F14BC14FF14CC147
:104AC00050F14DC151F14EC152F157C159F158C188
:104AD0005AF1079470EC25F0A0EC0EF09AEF2AF052
:104AE00066C100F167C101F168C102F169C103F15A
:104AF000010120EC31F0E3EC2EF00401630E826F33
:104B000096EC0EF004012C0E826F96EC0EF04FC165
:104B100000F150C101F151C102F152C103F1010193
:104B200020EC31F0E3EC2EF00401660E826F96EC7F
:104B30000EF004012C0E826F96EC0EF097EC31F023
:104B400059C100F15AC101F1010120EC31F0E3EC4F
:104B50002EF00401740E826F96EC0EF0120010829B
:104B60000401530E826F96EC0EF004012C0E826F3E
:104B700096EC0EF083C32AF184C32BF185C32CF18C
:104B800086C32DF187C32EF188C32FF189C330F17D
:104B90008AC331F18BC332F18CC333F10101E5ECEF
:104BA00031F05CEC31F000C166F101C167F102C186
:104BB00068F103C169F18EC32AF18FC32BF190C351
:104BC0002CF191C32DF192C32EF193C32FF194C315
:104BD00030F195C331F196C332F197C333F101013E
:104BE000E5EC31F05CEC31F000C14FF101C150F166
:104BF00002C151F103C152F1D8EC31F099C32FF148
:104C00009AC330F19BC331F19CC332F19DC333F1A0
:104C10000101E5EC31F05CEC31F000C159F101C16A
:104C20005AF170EC25F004012C0E826F96EC0EF018
:104C30002AEF26F0118E1CA002D01CAE108C1BBED9
:104C400002D01BA4108E03018251520A02E10F828E
:104C500001D00F928251750A02E1108401D01094A4
:104C60008251550A02E1108601D010968351310A13
:104C700003E11382138402D013921394030183512E
:104C8000660A01E056D00401660E826F96EC0EF0C3
:104C900004012C0E826F96EC0EF06EEC23F020ECEB
:104CA00031F02AC182F40401300E822796EC0EF016
:104CB0002BC182F40401300E822796EC0EF02CC139
:104CC00082F40401300E822796EC0EF02DC182F49E
:104CD0000401300E822796EC0EF02EC182F40401FE
:104CE000300E822796EC0EF02FC182F40401300EB4
:104CF000822796EC0EF030C182F40401300E822738
:104D000096EC0EF031C182F40401300E822796EC4D
:104D10000EF032C182F40401300E822796EC0EF0C0
:104D200033C182F40401300E822796EC0EF098EF26
:104D30002AF011A003D011A401D01084078410B26E
:104D400003EF27F010A4E7EF26F0BAC166F1BBC16C
:104D500067F1BCC168F1BDC169F1BEC16AF1BFC1F3
:104D60006BF1C0C16CF1C1C16DF1C2C16EF1C3C1C3
:104D70006FF1C4C170F1C5C171F1C6C172F1C7C193
:104D800073F1C8C174F1C9C175F1CAC176F1CBC163
:104D900077F1CCC178F1CDC179F1CEC17AF1CFC133
:104DA0007BF1D0C17CF1D1C17DF1D2C17EF1D3C103
:104DB0007FF1D4C180F1D5C181F1D6C182F1D7C1D3
:104DC00083F1D8C184F1D9C185F1EFEF26F062C13A
:104DD00066F163C167F164C168F165C169F1BAC187
:104DE00086F1BBC187F1BCC188F1BDC189F14BC15E
:104DF0004FF14CC150F14DC151F14EC152F157C16B
:104E000059F158C15AF107940FA025EF27F001017D
:104E1000966712EF27F0976712EF27F0986712EF67
:104E200027F0996716EF27F025EF27F071EC22F0B5
:104E300096C104F197C105F198C106F199C107F136
:104E400082EC30F003BF5EEF2AF071EC22F001013A
:104E5000000E046F000E056F010E066F000E076F47
:104E6000B3EC30F011A02AD011A228D020EC31F000
:104E7000296701D005D004012D0E826F96EC0EF04B
:104E800030C182F40401300E822796EC0EF031C15D
:104E900082F40401300E822796EC0EF032C182F4C7
:104EA0000401300E822796EC0EF033C182F4040127
:104EB000300E822796EC0EF0A0EC0EF012A8C5D0B2
:104EC00012981DC01EF01E3A1E42070E1E1600014B
:104ED0001E50000AD8B4F1EF27F000011E50010A5D
:104EE000D8B47DEF27F000011E50020AD8B47BEF42
:104EF00027F023EF28F023EF28F097EC31F02DC0B6
:104F000001F12EC000F1D89001330033D890013365
:104F100000330101630E046F000E056F000E066F73
:104F2000000E076FB3EC30F0280E046F000E056F13
:104F3000000E066F000E076F82EC30F000C130F0FB
:104F400097EC31F02BC001F1019F019D2CC000F1C5
:104F50000101A40E046F000E056F000E066F000E17
:104F6000076FB3EC30F000C12FF000C104F101C1B4
:104F700005F102C106F103C107F1640E006F000ED6
:104F8000016F000E026F000E036F82EC30F0050E11
:104F9000046F000E056F000E066F000E076FB3EC76
:104FA00030F000C104F101C105F102C106F103C1F5
:104FB00007F197EC31F030C000F182EC30F000C125
:104FC00031F031C0E8FF050F305C03E78A8423EF3E
:104FD00028F031C0E8FF0A0F305C01E68A9423EF25
:104FE00028F000C124F101C125F102C126F103C15D
:104FF00027F197EC31F09DEC31F01D501F0BE8CFFD
:1050000000F10101640E046F000E056F000E066FC3
:10501000000E076F93EC30F024C104F125C105F1B7
:1050200026C106F127C107F182EC30F003BF02D0A0
:105030008A9401D08A8424C100F125C101F126C1DE
:1050400002F127C103F19AEF2AF000C124F101C156
:1050500025F102C126F103C127F110AE4DD0109EFB
:1050600000C108F101C109F102C10AF103C10BF14C
:1050700020EC31F030C1E2F131C1E3F132C1E4F1B1
:1050800033C1E5F108C100F109C101F10AC102F122
:105090000BC103F101016C0E046F070E056F000ECA
:1050A000066F000E076F82EC30F003BF04D00101E1
:1050B000550EE66F1CD008C100F109C101F10AC10B
:1050C00002F10BC103F10101A40E046F060E056F7E
:1050D000000E066F000E076F82EC30F003BF04D0A5
:1050E00001017F0EE66F03D00101FF0EE66F1F8EF8
:1050F00011AE5EEF2AF0119E24C100F125C101F12D
:1051000026C102F127C103F111A005D011A203D0DD
:105110000FB05EEF2AF010A495EF28F00401750E91
:10512000826F96EC0EF09AEF28F00401720E826FF7
:1051300096EC0EF004012C0E826F96EC0EF020EC33
:1051400031F02967A9EF28F00401200E826FACEF3F
:1051500028F004012D0E826F96EC0EF030C182F41F
:105160000401300E822796EC0EF031C182F4040166
:10517000300E822796EC0EF004012E0E826F96EC14
:105180000EF032C182F40401300E822796EC0EF04C
:1051900033C182F40401300E822796EC0EF0040134
:1051A0006D0E826F96EC0EF004012C0E826F96EC61
:1051B0000EF04FC100F150C101F151C102F152C1D5
:1051C00003F1010120EC31F0E3EC2EF00401480E74
:1051D000826F96EC0EF004017A0E826F96EC0EF060
:1051E00004012C0E826F96EC0EF066C100F167C1CF
:1051F00001F168C102F169C103F1010120EC31F054
:10520000E3EC2EF00401630E826F96EC0EF00401C5
:105210002C0E826F96EC0EF066C100F167C101F1B1
:1052200068C102F169C103F101010A0E046F000EA9
:10523000056F000E066F000E076F93EC30F0000E46
:10524000046F120E056F000E066F000E076FB3ECB1
:1052500030F020EC31F02AC182F40401300E8227B4
:1052600096EC0EF02BC182F40401300E822796ECEE
:105270000EF02CC182F40401300E822796EC0EF061
:105280002DC182F40401300E822796EC0EF02EC15F
:1052900082F40401300E822796EC0EF02FC182F4C6
:1052A0000401300E822796EC0EF030C182F4040126
:1052B000300E822796EC0EF004012E0E826F96ECD3
:1052C0000EF031C182F40401300E822796EC0EF00C
:1052D00032C182F40401300E822796EC0EF033C105
:1052E00082F40401300E822796EC0EF00401730E56
:1052F000826F96EC0EF004012C0E826F96EC0EF08D
:1053000097EC31F059C100F15AC101F1C4EC2BF016
:1053100013A2DAEF29F004012C0E826F96EC0EF046
:1053200086C166F187C167F188C168F189C169F1F9
:1053300071EC22F00101000E046F000E056F010EEA
:10534000066F000E076FB3EC30F020EC31F02967E8
:10535000AFEF29F00401200E826FB2EF29F00401B3
:105360002D0E826F96EC0EF030C182F40401300EE7
:10537000822796EC0EF031C182F40401300E8227B0
:1053800096EC0EF004012E0E826F96EC0EF032C1F8
:1053900082F40401300E822796EC0EF033C182F4C1
:1053A0000401300E822796EC0EF004016D0E826F20
:1053B00096EC0EF003018351460A01E007D0040188
:1053C0002C0E826F96EC0EF059EC24F013A40DEF26
:1053D0002AF004012C0E826F96EC0EF013ACFBEF5A
:1053E00029F00401500E826F96EC0EF0139C139876
:1053F000139A0DEF2AF013AE08EF2AF00401460EBF
:10540000826F96EC0EF0139E1398139A0DEF2AF00C
:105410000401530E826F96EC0EF037B024EF2AF0A1
:1054200004012C0E826F96EC0EF08BB01FEF2AF069
:105430000401440E826F96EC0EF024EF2AF0040172
:10544000530E826F96EC0EF00FB22AEF2AF00FA0E7
:105450005CEF2AF004012C0E826F96EC0EF0200E09
:10546000F86EF76AF66A04010900F5CF82F496EC4B
:105470000EF00900F5CF82F496EC0EF00900F5CF9E
:1054800082F496EC0EF00900F5CF82F496EC0EF063
:105490000900F5CF82F496EC0EF00900F5CF82F406
:1054A00096EC0EF00900F5CF82F496EC0EF00900B0
:1054B000F5CF82F496EC0EF0A0EC0EF00F90109E5B
:1054C00012989AEF2AF00401630E826F96EC0EF0A8
:1054D00004012C0E826F96EC0EF0A0EC2AF0040171
:1054E0002C0E826F96EC0EF013EC2BF004012C0EB8
:1054F000826F96EC0EF08FEC2BF004012C0E826F75
:1055000096EC0EF00101F80E006FCD0E016F660EE5
:10551000026F030E036FB5EC2AF004012C0E826FAC
:1055200096EC0EF0A5EC2BF0A0EC0EF09AEF2AF022
:10553000A0EC0EF00301C26B07901092A9EF2DF0C2
:10554000D8900E0E64EC0BF0E8CF00F10F0E64EC77
:105550000BF0E8CF01F1100E64EC0BF0E8CF02F194
:10556000110E64EC0BF0E8CF03F10101000E046FA3
:10557000000E056F010E066F000E076FB3EC30F0E2
:1055800020EC31F02AC182F40401300E822796EC1F
:105590000EF02BC182F40401300E822796EC0EF03F
:1055A0002CC182F40401300E822796EC0EF02DC13E
:1055B00082F40401300E822796EC0EF02EC182F4A4
:1055C0000401300E822796EC0EF02FC182F4040104
:1055D000300E822796EC0EF030C182F40401300EBA
:1055E000822796EC0EF031C182F40401300E82273E
:1055F00096EC0EF004012E0E826F96EC0EF032C186
:1056000082F40401300E822796EC0EF033C182F44E
:105610000401300E822796EC0EF004016D0E826FAD
:1056200096EC0EF01200120E64EC0BF0E8CF00F1D5
:10563000130E64EC0BF0E8CF01F1140E64EC0BF0E8
:10564000E8CF02F1150E64EC0BF0E8CF03F1010195
:105650000A0E046F000E056F000E066F000E076F36
:1056600093EC30F0000E046F120E056F000E066F03
:10567000000E076FB3EC30F020EC31F02AC182F459
:105680000401300E822796EC0EF02BC182F4040147
:10569000300E822796EC0EF02CC182F40401300EFD
:1056A000822796EC0EF02DC182F40401300E822781
:1056B00096EC0EF02EC182F40401300E822796EC97
:1056C0000EF02FC182F40401300E822796EC0EF00A
:1056D00030C182F40401300E822796EC0EF00401F2
:1056E0002E0E826F96EC0EF031C182F40401300E62
:1056F000822796EC0EF032C182F40401300E82272C
:1057000096EC0EF033C182F40401300E822796EC41
:105710000EF00401730E826F96EC0EF012000A0E6A
:1057200064EC0BF0E8CF00F10B0E64EC0BF0E8CF6B
:1057300001F10C0E64EC0BF0E8CF02F10D0E64ECFD
:105740000BF0E8CF03F1C4EF2BF0060E64EC0BF086
:10575000E8CF00F1070E64EC0BF0E8CF01F1080E82
:1057600064EC0BF0E8CF02F1090E64EC0BF0E8CF2B
:1057700003F1C4EF2BF0010197EC31F0078457C11E
:1057800000F158C101F107940101E80E046F800E89
:10579000056F000E066F000E076F93EC30F0000EE1
:1057A000046F040E056F000E066F000E076FB3EC5A
:1057B00030F0880E046F130E056F000E066F000E9A
:1057C000076F82EC30F00A0E046F000E056F000EBA
:1057D000066F000E076FB3EC30F020EC31F00101E2
:1057E0002967F8EF2BF00401200E826FFBEF2BF0FE
:1057F00004012D0E826F96EC0EF030C182F404018C
:10580000300E822796EC0EF031C182F40401300E86
:10581000822796EC0EF032C182F40401300E82270A
:1058200096EC0EF004012E0E826F96EC0EF033C152
:1058300082F40401300E822796EC0EF00401430E30
:10584000826F96EC0EF0120087C32AF188C32BF109
:1058500089C32CF18AC32DF18BC32EF18CC32FF198
:105860008DC330F18EC331F190C332F191C333F166
:105870000101296BE5EC31F05CEC31F00101000E27
:10588000046F000E056F010E066F000E076F93EC9C
:1058900030F00E0E0C6E00C10BF04DEC0BF00F0E45
:1058A0000C6E01C10BF04DEC0BF0100E0C6E02C132
:1058B0000BF04DEC0BF0110E0C6E03C10BF04DEC28
:1058C0000BF004017A0E826F96EC0EF004012C0EA0
:1058D000826F96EC0EF00401350E826F96EC0EF09E
:1058E00004012C0E826F96EC0EF0A0EC2AF047EF2C
:1058F00022F087C32AF188C32BF189C32CF18AC314
:105900002DF18BC32EF18CC32FF18DC330F18EC3DB
:1059100031F190C332F191C333F10101296BE5EC10
:1059200031F05CEC31F0880E046F130E056F000E41
:10593000066F000E076F87EC30F0000E046F040E48
:10594000056F000E066F000E076F93EC30F001013B
:10595000E80E046F800E056F000E066F000E076FD5
:10596000B3EC30F00A0E0C6E00C10BF04DEC0BF0F6
:105970000B0E0C6E01C10BF04DEC0BF00C0E0C6E0F
:1059800002C10BF04DEC0BF00D0E0C6E03C10BF0D1
:105990004DEC0BF004017A0E826F96EC0EF00401D0
:1059A0002C0E826F96EC0EF00401360E826F96EC90
:1059B0000EF004012C0E826F96EC0EF08FEC2BF0A3
:1059C00047EF22F087C32AF188C32BF189C32CF15A
:1059D0008AC32DF18BC32EF18CC32FF18DC330F10F
:1059E0008FC331F190C332F191C333F10101E5EC82
:1059F00031F05CEC31F0000E046F120E056F000EFA
:105A0000066F000E076F93EC30F001010A0E046F71
:105A1000000E056F000E066F000E076FB3EC30F03E
:105A2000120E0C6E00C10BF04DEC0BF0130E0C6E51
:105A300001C10BF04DEC0BF0140E0C6E02C10BF01B
:105A40004DEC0BF0150E0C6E03C10BF04DEC0BF092
:105A500004017A0E826F96EC0EF004012C0E826F18
:105A600096EC0EF00401370E826F96EC0EF00401F6
:105A70002C0E826F96EC0EF013EC2BF047EF22F019
:105A800087C32AF188C32BF189C32CF18AC32DF176
:105A90008BC32EF18CC32FF18DC330F18EC331F146
:105AA00090C332F191C333F10101296BE5EC31F080
:105AB0005CEC31F0880E046F130E056F000E066F5C
:105AC000000E076F87EC30F0000E046F040E056FB8
:105AD000000E066F000E076F93EC30F00101E80E28
:105AE000046F800E056F000E066F000E076FB3EC9B
:105AF00030F0060E0C6E00C10BF04DEC0BF0070EF3
:105B00000C6E01C10BF04DEC0BF0080E0C6E02C1D7
:105B10000BF04DEC0BF0090E0C6E03C10BF04DECCD
:105B20000BF004017A0E826F96EC0EF004012C0E3D
:105B3000826F96EC0EF00401380E826F96EC0EF038
:105B400004012C0E826F96EC0EF0A5EC2BF047EFC3
:105B500022F007A81CEF2EF00101800E006F1A0E34
:105B6000016F060E026F000E036F4BC104F14CC1B2
:105B700005F14DC106F14EC107F182EC30F003BFD3
:105B800062EF2EF0DDEC2EF04BC100F14CC101F1C3
:105B90004DC102F14EC103F107828FEC2FF018C105
:105BA00004F119C105F11AC106F11BC107F1F80E84
:105BB000006FCD0E016F660E026F030E036F82EC55
:105BC00030F00E0E0C6E00C10BF04DEC0BF00F0E12
:105BD0000C6E01C10BF04DEC0BF0100E0C6E02C1FF
:105BE0000BF04DEC0BF0110E0C6E03C10BF04DECF5
:105BF0000BF00784010197EC31F057C100F158C157
:105C000001F107940A0E0C6E00C10BF04DEC0BF085
:105C10000B0E0C6E01C10BF04DEC0BF00C0E0C6E6C
:105C200002C10BF04DEC0BF00D0E0C6E03C10BF02E
:105C30004DEC0BF062EF2EF007AA62EF2EF0078416
:105C4000010197EC31F057C100F158C101F10794FF
:105C5000060E0C6E00C10BF04DEC0BF0070E0C6E37
:105C600001C10BF04DEC0BF0080E0C6E02C10BF0F5
:105C70004DEC0BF0090E0C6E03C10BF04DEC0BF06C
:105C8000078462C100F163C101F164C102F165C121
:105C900003F10794120E0C6E00C10BF04DEC0BF0EB
:105CA000130E0C6E01C10BF04DEC0BF0140E0C6ECC
:105CB00002C10BF04DEC0BF0150E0C6E03C10BF096
:105CC0004DEC0BF00798079A0401805181197F0B66
:105CD0000DE09EA8FED714EE00F081517F0BE12667
:105CE000E750812B0F01AD6E64EF2EF005012F51AF
:105CF000000AD8B4A5EF2EF081BA8AEF2EF015B2C3
:105D0000A5EF2EF005012F51010AD8B4A3EF2EF014
:105D10009CEF2EF005012F51000AD8B45CEF39F04A
:105D200005012F51010AD8B4A3EF2EF0000116503F
:105D3000050AD8B45CEF39F081B8A5EF2EF0E0EC9D
:105D400032F0DEEC33F0F5EC38F0C4EF0DF018C1B2
:105D500000F119C101F11AC102F11BC103F1000EDA
:105D6000046F000E056F010E066F000E076FB3EC97
:105D700030F029A1D2EF2EF02051D8B4D2EF2EF07E
:105D800018C100F119C101F11AC102F11BC103F1DF
:105D9000000E046F000E056F0A0E066F000E076FEF
:105DA000B3EC30F01200010104510013055101134E
:105DB000065102130751031312000101186B196BEE
:105DC0001A6B1B6B12002AC182F40401300E822769
:105DD00096EC0EF02BC182F40401300E822796EC73
:105DE0000EF02CC182F40401300E822796EC0EF0E6
:105DF0002DC182F40401300E822796EC0EF02EC1E4
:105E000082F40401300E822796EC0EF02FC182F44A
:105E10000401300E822796EC0EF030C182F40401AA
:105E2000300E822796EC0EF031C182F40401300E60
:105E3000822796EC0EF032C182F40401300E8227E4
:105E400096EC0EF033C182F40401300E822796ECFA
:105E50000EF012002FC182F40401300E822796EC5E
:105E60000EF030C182F40401300E822796EC0EF061
:105E700031C182F40401300E822796EC0EF032C15B
:105E800082F40401300E822796EC0EF033C182F4C6
:105E90000401300E822796EC0EF01200060E216EE1
:105EA000060E226E060E236E212E54EF2FF0222EA8
:105EB00054EF2FF0232E54EF2FF08B84020E216E1F
:105EC000020E226E020E236E212E64EF2FF0222E80
:105ED00064EF2FF0232E64EF2FF08B941200FF0E4F
:105EE000226E22C023F0030E216E8B84212E75EFCB
:105EF0002FF0030E216E232E75EF2FF08B9422C00E
:105F000023F0030E216E212E83EF2FF0030E216E5E
:105F1000233E83EF2FF0222E71EF2FF012000101AC
:105F2000005305E1015303E1025301E1002B52EC60
:105F300030F097EC31F03951006F3A51016F420E59
:105F4000046F4B0E056F000E066F000E076F93EC8B
:105F500030F000C104F101C105F102C106F103C135
:105F600007F118C100F119C101F11AC102F11BC1F9
:105F700003F107B2C0EF2FF087EC30F0C2EF2FF043
:105F800082EC30F000C118F101C119F102C11AF11F
:105F900003C11BF1120097EC31F059C100F15AC155
:105FA00001F1060E64EC0BF0E8CF04F1070E64EC8F
:105FB0000BF0E8CF05F1080E64EC0BF0E8CF06F12A
:105FC000090E64EC0BF0E8CF07F182EC30F000C171
:105FD00024F101C125F102C126F103C127F1290EE7
:105FE000046F000E056F000E066F000E076F93EC36
:105FF00030F0EE0E046F430E056F000E066F000EBC
:10600000076F87EC30F024C104F125C105F126C1EA
:1060100006F127C107F193EC30F000C11CF101C17A
:106020001DF102C11EF103C11FF1120E64EC0BF051
:10603000E8CF04F1130E64EC0BF0E8CF05F1140E79
:1060400064EC0BF0E8CF06F1150E64EC0BF0E8CF32
:1060500007F10D0E006F000E016F000E026F000EB3
:10606000036F93EC30F0180E046F000E056F000EF6
:10607000066F000E076FB3EC30F01CC104F11DC1B8
:1060800005F11EC106F11FC107F187EC30F06A0E61
:10609000046F2A0E056F000E066F000E076F82EC6C
:1060A00030F01200BF0EFA6E200E3A6F396BD890A6
:1060B0000037013702370337D8B063EF30F03A2F9B
:1060C00058EF30F039073A070353D8B412000331C0
:1060D000070B80093F6F03390F0B010F396F80ECFD
:1060E0005FF0406F390580EC5FF0405D405F396BD9
:1060F0003F33D8B0392739333FA978EF30F04051DA
:10610000392712000101BCEC31F0D8B012000101B6
:1061100003510719346F7FEC31F0D8900751031900
:1061200034AF800F12000101346BA3EC31F0D8A022
:10613000B9EC31F0D8B012008EEC31F097EC31F0C0
:106140001F0E366FCFEC31F00B35D8B07FEC31F04D
:10615000D8A00335D8B01200362FA2EF30F034B1FA
:10616000A6EC31F012000101346B04510511061147
:1061700007110008D8A0A3EC31F0D8A0B9EC31F099
:10618000D8B01200086B096B0A6B0B6BCFEC31F0C7
:106190001F0E366FCFEC31F007510B5DD8A4DDEF49
:1061A00030F006510A5DD8A4DDEF30F00551095DED
:1061B000D8A4DDEF30F00451085DD8A0F0EF30F046
:1061C0000451085F0551D8A0053D095F0651D8A0CC
:1061D000063D0A5F0751D8A0073D0B5FD8900081AC
:1061E000362FCAEF30F034B1A6EC31F0346BA3ECAB
:1061F00031F0D890D3EC31F007510B5DD8A40DEFFE
:1062000031F006510A5DD8A40DEF31F00551095D5A
:10621000D8A40DEF31F00451085DD8A01CEF31F087
:10622000003F1CEF31F0013F1CEF31F0023F1CEF4B
:1062300031F0032BD8B4120034B1A6EC31F01200C7
:106240000101346BA3EC31F0D8B01200D8EC31F07E
:10625000200E366F003701370237033711EE33F067
:106260000A0E376FE7360A0EE75CD8B0E76EE552E4
:10627000372F32EF31F0362F2AEF31F034B1298148
:10628000D8901200D8EC31F0200E366F003701376D
:106290000237033711EE33F00A0E376FE7360A0E76
:1062A000E75CD8B0E76EE552372F4EEF31F0362F6E
:1062B00046EF31F0D890120001010A0E346F200E23
:1062C000366F11EE29F03451376F0A0ED890E6522E
:1062D000D8B0E726E732372F67EF31F003330233C8
:1062E00001330033362F61EF31F0E750FF0FD8A0B4
:1062F0000335D8B0120029B1A6EC31F012000451D8
:1063000000270551D8B0053D01270651D8B0063DFC
:1063100002270751D8B0073D032712000051086F2C
:106320000151096F02510A6F03510B6F12000101F5
:10633000006B016B026B036B12000101046B056BB8
:10634000066B076B12000335D8A012000351800BB7
:10635000001F011F021F031F003FB6EF31F0013F76
:10636000B6EF31F0023FB6EF31F0032B342B0325AB
:1063700012000735D8A012000751800B041F051F1B
:10638000061F071F043FCCEF31F0053FCCEF31F083
:10639000063FCCEF31F0072B342B072512000037D6
:1063A000013702370337083709370A370B3712002E
:1063B0000101296B2A6B2B6B2C6B2D6B2E6B2F6BBA
:1063C000306B316B326B336B120001012A510F0BB2
:1063D0002A6F2B510F0B2B6F2C510F0B2C6F2D5144
:1063E0000F0B2D6F2E510F0B2E6F2F510F0B2F6F89
:1063F00030510F0B306F31510F0B316F32510F0B8A
:10640000326F33510F0B336F120000C124F101C101
:1064100025F102C126F103C127F104C100F105C134
:1064200001F106C102F107C103F124C104F125C144
:1064300005F126C106F127C107F1120010A806D008
:106440008994000EC76E220EC66E05D08984000E98
:10645000C76E220EC66E050EE82EFED7120010A8DB
:1064600002D0898401D08994050EE82EFED712004F
:106470001EEC32F09E96C69E000EC96EFF0E9EB6B2
:1064800002D0E82EFCD79E96C69E000EC96EFF0E67
:106490009EB602D0E82EFCD7C9CFAFF59E96C69E19
:1064A000000EC96EFF0E9EB602D0E82EFCD7C9CFF3
:1064B000B0F59E96C69E000EC96EFF0E9EB602D027
:1064C000E82EFCD7C9CFB1F59E96C69E000EC96EC8
:1064D000FF0E9EB602D0E82EFCD7C9CFB2F59E962D
:1064E000C69E000EC96EFF0E9EB602D0E82EFCD7E7
:1064F000C9CFB3F59E96C69E000EC96EFF0E9EB61E
:1065000002D0E82EFCD7C9CFB4F59E96C69E000EE9
:10651000C96EFF0E9EB602D0E82EFCD7C9CFB5F5E6
:106520002FEC32F012001EEC32F09E96C69E800ECA
:10653000C96EFF0E9EB602D0E82EFCD79E96C69E70
:10654000AFC5C9FFFF0E9EB602D0E82EFCD79E96BF
:10655000C69EB0C5C9FFFF0E9EB602D0E82EFCD77E
:106560009E96C69EB1C5C9FFFF0E9EB602D0E82E0C
:10657000FCD79E96C69EB2C5C9FFFF0E9EB602D03E
:10658000E82EFCD79E96C69EB3C5C9FFFF0E9EB6E9
:1065900002D0E82EFCD79E96C69EB4C5C9FFFF0E5A
:1065A0009EB602D0E82EFCD79E96C69EB5C5C9FF02
:1065B000FF0E9EB602D0E82EFCD72FEC32F0120070
:1065C0001EEC32F09E96C69E070EC96EFF0E9EB65A
:1065D00002D0E82EFCD79E96C69E000EC96EFF0E16
:1065E0009EB602D0E82EFCD7C9CFAFF59E96C69EC8
:1065F000000EC96EFF0E9EB602D0E82EFCD7C9CFA2
:10660000B0F59E96C69E000EC96EFF0E9EB602D0D5
:10661000E82EFCD7C9CFB1F59E96C69E000EC96E76
:10662000FF0E9EB602D0E82EFCD7C9CFB2F52FECF4
:1066300032F01EEC32F09E96C69E25C0C9FFFF0EBA
:106640009EB602D0E82EFCD79E96C69E000EC96E5E
:10665000FF0E9EB602D0E82EFCD7C9CFB6F52FECC0
:1066600032F012001EEC32F09E96C69E870EC96E66
:10667000FF0E9EB602D0E82EFCD79E96C69EAFC5F2
:10668000C9FFFF0E9EB602D0E82EFCD79E96C69E8E
:10669000B0C5C9FFFF0E9EB602D0E82EFCD79E966D
:1066A000C69EB1C5C9FFFF0E9EB602D0E82EFCD72C
:1066B0009E96C69EB2C5C9FFFF0E9EB602D0E82EBA
:1066C000FCD72FEC32F01EEC32F09E96C69E26C010
:1066D000C9FFFF0E9EB602D0E82EFCD79E96C69E3E
:1066E000B6C5C9FFFF0E9EB602D0E82EFCD72FEC30
:1066F00032F012001EEC32F09E96C69E870EC96ED6
:10670000FF0E9EB602D0E82EFCD79E96C69E000EC7
:10671000C96EFF0E9EB602D0E82EFCD79E96C69E8E
:10672000800EC96EFF0E9EB602D0E82EFCD79E9654
:10673000C69E800EC96EFF0E9EB602D0E82EFCD714
:106740009E96C69E800EC96EFF0E9EB602D0E82EA3
:10675000FCD72FEC32F012001EEC32F09E96C69E53
:10676000870EC96EFF0E9EB602D0E82EFCD79E960D
:10677000C69E000EC96EFF0E9EB602D0E82EFCD754
:106780009E96C69E000EC96EFF0E9EB602D0E82EE3
:10679000FCD79E96C69E800EC96EFF0E9EB602D096
:1067A000E82EFCD79E96C69E800EC96EFF0E9EB642
:1067B00002D0E82EFCD72FEC32F0120010A817D030
:1067C0001EEC32F09E96C69E8F0EC96EFF0E9EB6D0
:1067D00002D0E82EFCD79E96C69E000EC96EFF0E14
:1067E0009EB602D0E82EFCD72FEC32F01200E0EC7F
:1067F00032F0120010A82DD01EEC32F09E96C69EEC
:1068000026C0C9FFFF0E9EB602D0E82EFCD79E968A
:10681000C69E450EC96EFF0E9EB602D0E82EFCD76E
:106820002FEC32F01EEC32F09E96C69E8F0EC96E93
:10683000FF0E9EB602D0E82EFCD79E96C69E000E96
:10684000C96EFF0E9EB602D0E82EFCD72FEC32F0B8
:1068500012001EEC32F09E96C69E26C0C9FFFF0EA7
:106860009EB602D0E82EFCD79E96C69E010EC96E3B
:10687000FF0E9EB602D0E82EFCD72FEC32F01EECB5
:1068800032F09E96C69E910EC96EFF0E9EB602D045
:10689000E82EFCD79E96C69EA50EC96EFF0E9EB62C
:1068A00002D0E82EFCD72FEC32F012001EEC32F0B2
:1068B0009E96C69E26C0C9FFFF0E9EB602D0E82E49
:1068C000FCD79E96C69E810EC96EFF0E9EB602D064
:1068D000E82EFCD72FEC32F012001EEC32F09E9620
:1068E000C69E26C0C9FFFF0E9EB602D0E82EFCD77A
:1068F0009E96C69E010EC96EFF0E9EB602D0E82E71
:10690000FCD72FEC32F012001EEC32F09E96C69EA1
:10691000910EC96EFF0E9EB602D0E82EFCD79E9651
:10692000C69EA50EC96EFF0E9EB602D0E82EFCD7FD
:106930002FEC32F012001EEC32F09E96C69E910EA5
:10694000C96EFF0E9EB602D0E82EFCD79E96C69E5C
:10695000000EC96EFF0E9EB602D0E82EFCD72FECBB
:1069600032F012000501256B266B276B286B899A84
:10697000400EC76E200EC66E9E96C69E030EC96E52
:10698000FF0E9EB602D0E82EFCD79E96C69E27C567
:10699000C9FFFF0E9EB602D0E82EFCD79E96C69E7B
:1069A00026C5C9FFFF0E9EB602D0E82EFCD79E96E4
:1069B000C69E25C5C9FFFF0E9EB602D0E82EFCD7A5
:1069C0009E96C69EC952FF0E9EB602D0E82EFCD7F8
:1069D000898A0F01C950FF0A01E1120005012E51F9
:1069E000130A05E005012E51170A0CE012000501FB
:1069F000F00E256FFF0E266F0F0E276F000E286F0B
:106A00000BEF35F00501F00E256FFF0E266FFF0E20
:106A1000276F000E286F899A400EC76E200EC66E33
:106A20009E96C69E030EC96EFF0E9EB602D0E82E3D
:106A3000FCD79E96C69E27C5C9FFFF0E9EB602D004
:106A4000E82EFCD79E96C69E26C5C9FFFF0E9EB6B1
:106A500002D0E82EFCD79E96C69E25C5C9FFFF0E24
:106A60009EB602D0E82EFCD79E96C69EC952FF0E57
:106A70009EB602D0E82EFCD7898A0F01C950FF0AC2
:106A80001DE005012E51130A05E005012E51170ADC
:106A90000BE012000501000E256F000E266F100E90
:106AA000276F000E286F12000501000E256F000EE3
:106AB000266F000E276F010E286F12000501256B4F
:106AC000266B276B286B05012E51130A05E0050183
:106AD0002E51170A0CE012000501000E216F000E66
:106AE000226F080E236F000E246F80EF35F0050132
:106AF000000E216F000E226F800E236F000E246F98
:106B000021C500F122C501F123C502F124C503F11D
:106B100025C504F126C505F127C506F128C507F1ED
:106B2000D3EC2EF000C125F501C126F502C127F5F1
:106B300003C128F5899A400EC76E200EC66E9E9638
:106B4000C69E030EC96EFF0E9EB602D0E82EFCD77D
:106B50009E96C69E27C5C9FFFF0E9EB602D0E82EA0
:106B6000FCD79E96C69E26C5C9FFFF0E9EB602D0D4
:106B7000E82EFCD79E96C69E25C5C9FFFF0E9EB681
:106B800002D0E82EFCD79E96C69EC952FF0E9EB636
:106B900002D0E82EFCD7898AC950FF0A08E104C157
:106BA00025F505C126F506C127F507C128F5D890BA
:106BB000050124332333223321332151F00B216F7C
:106BC00005012167EBEF35F02267EBEF35F0236726
:106BD000EBEF35F0246780EF35F00501100E252727
:106BE000E86A2623E86A2723E86A28231200E86A6D
:106BF00005012E51130A06E005012E51170A0BE07C
:106C0000020E120005012851000A03E12751F00B82
:106C100007E0010E120005012851000A01E0010EF3
:106C2000120029C500F12AC501F12BC502F12CC5BE
:106C300003F125C504F126C505F127C506F128C5D0
:106C400007F182EC30F003BF1200F7EC35F0D8A466
:106C500089EF36F0899A400EC76E200EC66E9E965A
:106C6000C69E060EC96EFF0E9EB602D0E82EFCD759
:106C7000898A899A9E96C69E020EC96EFF0E9EB69E
:106C800002D0E82EFCD79E96C69E27C5C9FFFF0EF0
:106C90009EB602D0E82EFCD79E96C69E26C5C9FF9A
:106CA000FF0E9EB602D0E82EFCD79E96C69E25C546
:106CB000C9FFFF0E9EB602D0E82EFCD79E96C69E58
:106CC000000EC96EFF0E9EB602D0E82EFCD7898A50
:106CD000899A9E96C69E050EC96EFF0E9EB602D07C
:106CE000E82EFCD79E96C69EC952FF0E9EB602D0D5
:106CF000E82EFCD7C9B072EF36F0898A0501100E74
:106D00002527E86A2623E86A2723E86A282311EF63
:106D100036F01200899A400EC76E200EC66E9E96FF
:106D2000C69E060EC96EFF0E9EB602D0E82EFCD798
:106D3000898A899A9E96C69EC70EC96EFF0E9EB618
:106D400002D0E82EFCD7898A0501256B266B276BBC
:106D5000286B1200899A400EC76E200EC66E9E9652
:106D6000C69E050EC96EFF0E9EB602D0E82EFCD759
:106D70009E96C69EC952FF0E9EB602D0E82EFCD744
:106D8000C9CF37F5898A1200899A400EC76E200E46
:106D9000C66E9E96C69EB90EC96EFF0E9EB602D0F6
:106DA000E82EFCD7898A1200899A400EC76E200E01
:106DB000C66E9E96C69EAB0EC96EFF0E9EB602D0E4
:106DC000E82EFCD7898AFF0EE82EFED71200F7ECDA
:106DD00035F0D8A41200899A400EC76E200EC66EF8
:106DE0009E96C69E030EC96EFF0E9EB602D0E82E7A
:106DF000FCD79E96C69E27C5C9FFFF0E9EB602D041
:106E0000E82EFCD79E96C69E26C5C9FFFF0E9EB6ED
:106E100002D0E82EFCD79E96C69E25C5C9FFFF0E60
:106E20009EB602D0E82EFCD79E96C69EC952FF0E93
:106E30009EB602D0E82EFCD7898A0F01C950FF0AFE
:106E4000D8A466EF38F00501FE0E376F0501FF0E7E
:106E5000536FFF0E546FFF0E556FFF0E566F15A642
:106E60003799158638EC32F0AFC538F5B0C539F52D
:106E7000B1C53AF5B2C53BF5B3C53CF5B4C53DF572
:106E8000B5C53EF50784BAC166F1BBC167F1BCC1A7
:106E900068F1BDC169F14BC14FF14CC150F14DC119
:106EA00051F14EC152F157C159F158C15AF1000187
:106EB0001650010AD8B46BEF37F000011650020AE1
:106EC000D8B490EF37F000011650040AD8B4B5EFEB
:106ED00037F066EF38F00501476B486B496B4A6B3A
:106EE00005014B6B4C6B4D6B4E6B05014F6B506B43
:106EF000516B526B8BA0379B71EC22F000C1DAF121
:106F000001C1DBF102C1DCF103C1DDF100C13FF5DC
:106F100001C140F502C141F503C142F5D4EF37F09C
:106F20000501476B486B496B4A6B05014B6B4C6B1A
:106F30004D6B4E6B05014F6B506B516B526B71EC8F
:106F400022F000C1DAF101C1DBF102C1DCF103C1C1
:106F5000DDF16EEC23F000C147F501C148F502C137
:106F600049F503C14AF566EF38F0379BDAC13FF5C2
:106F7000DBC140F5DCC141F5DDC142F571EC22F029
:106F800000C14BF501C14CF502C14DF503C14EF5F1
:106F90006EEC23F000C14FF501C150F502C151F56F
:106FA00003C152F5D4EF37F005016167DFEF37F029
:106FB0006267DFEF37F06367DFEF37F06467E3EFB7
:106FC00037F0F8EF37F0DAC100F1DBC101F1DCC1D5
:106FD00002F1DDC103F161C504F162C505F163C5CC
:106FE00006F164C507F182EC30F003BF66EF38F0BC
:106FF00059C143F55AC144F5B9C545F50501110E0E
:10700000326F899A400EC76E200EC66E9E96C69E3F
:10701000060EC96EFF0E9EB602D0E82EFCD7898AF6
:10702000899A9E96C69E020EC96EFF0E9EB602D02B
:10703000E82EFCD79E96C69E27C5C9FFFF0E9EB6BA
:1070400002D0E82EFCD79E96C69E26C5C9FFFF0E2D
:107050009EB602D0E82EFCD79E96C69E25C5C9FFD7
:10706000FF0E9EB602D0E82EFCD725EE37F0322F69
:1070700002D046EF38F09E96C69EDECFC9FFFF0EC7
:107080009EB602D0E82EFCD737EF38F0898A899A6D
:107090009E96C69E050EC96EFF0E9EB602D0E82EC5
:1070A000FCD79E96C69EC952FF0E9EB602D0E82E11
:1070B000FCD7C9B051EF38F0898A0501100E252799
:1070C000E86A2623E86A2723E86A282315900794AC
:1070D000120021C500F122C501F123C502F124C52A
:1070E00003F1899A400EC76E200EC66E9E96C69E0C
:1070F0000B0EC96EFF0E9EB602D0E82EFCD79E96F0
:10710000C69E02C1C9FFFF0E9EB602D0E82EFCD774
:107110009E96C69E01C1C9FFFF0E9EB602D0E82E04
:10712000FCD79E96C69E00C1C9FFFF0E9EB602D038
:10713000E82EFCD79E96C69EC952FF0E9EB602D080
:10714000E82EFCD725EE37F00501100E326F9E9623
:10715000C69EC952FF0E9EB602D0E82EFCD7C9CFFC
:10716000DEFF322FA7EF38F0898A1200899A400E8D
:10717000C76E200EC66E9E96C69E900EC96EFF0EFE
:107180009EB602D0E82EFCD79E96C69E000EC96E13
:10719000FF0E9EB602D0E82EFCD79E96C69E000E2D
:1071A000C96EFF0E9EB602D0E82EFCD79E96C69EF4
:1071B000000EC96EFF0E9EB602D0E82EFCD79E963A
:1071C000C69EC952FF0E9EB602D0E82EFCD7C9CF8C
:1071D0002DF59E96C69EC952FF0E9EB602D0E82E91
:1071E000FCD7C9CF2EF5898A120038EC32F00501A0
:1071F0002F51010A5FE005012F51020A16E0050137
:107200002F51030A19E005012F51040A24E005015A
:107210002F51050A2BE005012F51060A39E005011F
:107220002F51070A3FE05AEF39F0602F58EF39F03D
:107230005FC560F55AEF39F0B0C500F101010F0EDE
:10724000001701010051000A35E001010051050A53
:1072500031E058EF39F0B0C500F101010F0E001711
:1072600001010051000A26E058EF39F00501B05144
:10727000000A20E00501B051150A1CE00501B051DB
:10728000300A18E00501B051450A14E058EF39F012
:107290000501B051000A0EE00501B051300A0AE0C4
:1072A00058EF39F00501B051000A04E058EF39F009
:1072B00015901200158012008B904EEC2FF0B9C57E
:1072C000E8FFD70802E34EEC2FF0B9C5E8FFC80885
:1072D00002E34EEC2FF0B9C5E8FFB90802E34EEC2B
:1072E0002FF0B9C5E8FFAA0802E34EEC2FF0B9C5AC
:1072F000E8FF9B0802E34EEC2FF0C4EC36F0F29C62
:10730000F29E8B94C69AC2909482948C720ED36E25
:10731000D3A4FED789968A909390F29AF2949D9086
:107320009E909D929E92F298F292DEEC33F0FF0EC8
:10733000E8CF00F0E82EFED7002EFCD7F290F286C0
:10734000815081A8A6EF39F0F29E0300700ED36E33
:10735000F296F290158403806FEC2FF09AEF0BF009
:10BF0000E844F926000C160C2B0C3F0C520C640C68
:10BF1000760C860C960CA50CB30CC10CCF0CDC0C6B
:06BF2000E80CF40C000C1B
:0200000400F00A
:0100C800FE39
:00000001FF
